:100000000C9472030C9430190C9409190C949A03F3
:100010000C949A030C949A030C949A030C94BB17B7
:100020000C949A030C949A030C949A030C94B607BC
:100030000C949A030C949A030C949A030C949A03CC
:100040000C94BF180C949A030C9430170C940A1754
:100050000C949A030C949A030C949A030C949A03AC
:100060000C9457190C949A035D2A892AA52ABE2A52
:10007000EE2A182B342B4E414E494E495459494EC5
:1000800046CDCCCC3D0AD7233C17B7D13877CC2B03
:10009000329595E6241FB14F0A000020410000C8A8
:1000A0004200401C4620BCBE4CCA1B0E5AAEC59D29
:1000B0007441644E6F76656120202020202032300C
:1000C0003138286329002D2D2D0047656967657239
:1000D0002D4D756C6C6572206465766963650043AF
:1000E0002D474D2076004E6574776F726B206469E2
:1000F0007361626C656400206279204C6175726581
:100100006E74202F2041644E6F766561202D203261
:100110003031382863290A54797065203F20666F92
:10012000722075736167650A00432D474D20760084
:1001300053454C45435420746F207475726E2D6F77
:100140006666005455524E204F464620444953504F
:100150004C41593F0053454C45435420746F207324
:1001600061766500536176656421005341564520F0
:10017000544F20454550524F4D3F004E4554574F28
:10018000524B2041435449564154494F4E3A004C3A
:10019000494748542054494D454F55543A004F66FD
:1001A00066004F6E00534F554E443A0053454C4540
:1001B000435420746F20636C65617200436C656109
:1001C0007265642100434C45415220434F554E54C3
:1001D0004552533F0053454C45435420746F2051C2
:1001E000756974004D454E553A0041644E6F766511
:1001F00061287229202D20323031382863290043AC
:100200002D474D2076002E002E002E005376723D95
:10021000004E2F41004465763D004E4554574F52E5
:100220004B2049503A002043504D2000416C6172F0
:100230006D2054687265733D20002056200054756F
:10024000626520482E562E20203D200054756265A0
:1002500020466163746F723D200052653A00537608
:100260003A2000444F53452000434F554E545320ED
:10027000203A20005F5F5F5F5F5F0044414E47456B
:10028000522100454D455247454E4359004352497E
:10029000544943414C0048494748204C4556454C39
:1002A000005761726E696E670053616665004E6F3C
:1002B000726D616C004176673A0043504D3A004DD3
:1002C00061783A0053763A00205600486967682002
:1002D000566F6C746167653D20005741524E494E20
:1002E000473A2000496E76616C696421004F4B00EB
:1002F000436F6E6E656374696F6E3A20636C6F73E3
:10030000650D0A0D0A00436F6E74656E742D547985
:1003100070653A20746578742F706C61696E0D0A8F
:1003200000436F6E74656E742D547970653A206168
:1003300070706C69636174696F6E2F6A736F6E0D94
:100340000A00485454502F312E3120323030204F83
:100350004B0D0A0053454E44206661696C6564008C
:10036000636F6D706C65746564210020485454504F
:100370002F312E300D0A003F0047455420005365B1
:100380006E64696E672043504D2F41564720766159
:100390006C75657320004661696C65642100432DAE
:1003A000474D20436F756E7465722049503A2000A6
:1003B000290A00202800467265652028422920204D
:1003C0003A20000A55534147453A0A202046414306
:1003D000544F523D7878782E780A202048563D7840
:1003E0007878205B302D3235355D0A2020414C4134
:1003F000524D3D787878782043504D0A2020524560
:1004000053455420636F756E746572730A0A202019
:10041000424545503D4F4E2F4F46460A20205449F5
:100420004D454F55543D7878780A20204C43443D43
:100430004F4E2F4F46460A0A20204E4554574F52E2
:100440004B3D4F4E2F4F46460A20204D41433D78AD
:1004500078783A7878783A7878783A7878783A7814
:1004600078783A7878780A20205345525645523D9C
:100470007878782E7878782E7878782E7878780A48
:10048000202055524C3D2F7878782F7878782E7030
:1004900068700A0A20204D454D4F52590A20204FBE
:1004A0005054494F4E530A2020454550524F4D0A53
:1004B000202056455253494F4E0A20204A534F4E52
:1004C0000A00220A097D0A7D0A7D00222C0A0909F8
:1004D0002274696D65223A202200222C0A09092221
:1004E00064617465223A2022002C0A092276657222
:1004F00073696F6E223A207B0A0909227265766958
:1005000073696F6E223A202200222C0A0922667239
:1005100065655F737461636B223A2000222C0A09BF
:100520002275726C223A2022002E002E002E00220C
:100530002C0A09227365727665725F6970223A200F
:1005400022004E2F41002C0A0922646576696365FA
:100550005F6970223A2022002C0A09226E657477A6
:100560006F726B223A20002C0A092274696D656F44
:100570007574223A20002C0A0922736F756E64226A
:100580003A20002C0A0922616C61726D223A200027
:100590002C0A09226876223A20002C0A0922766F5A
:1005A0006C74616765223A2000222C0A0922666178
:1005B00063746F72223A2000222C0A0922656C6152
:1005C00070736564223A20220009226465766963AB
:1005D000656964223A2022000922646573637269A6
:1005E0007074696F6E223A2022432D474D20434F8D
:1005F000554E544552222C0A0022706172616D736F
:10060000223A207B0A000A7D2C0A000922454C5020
:10061000223A20002C0A000922544F54223A20008A
:100620002C0A000922415647223A20002C0A0009D0
:10063000224D4158223A20002C0A00092243504DF5
:10064000223A20007B0A2264617461223A207B0AEC
:100650000000000000240027002A00000000002302
:100660000026002900000000080002010000030429
:1006700007000000000000000053454C4543542093
:10068000746F206D6F64696679004D6F6469667977
:10069000207573696E67205553422F4C414E0001FF
:1006A0000204081020408001020408102001020406
:1006B00008102000000000250028002B000404047E
:1006C00004040404040202020202020303030303FB
:1006D00003025361766520696E20454550524F4DA7
:1006E0000000813211241FBECFEFD8E0DEBFCDBFA6
:1006F00012E0A0E0B1E0EEE0F4E702C005900D9258
:10070000AE3DB107D9F726E0AEEDB2E001C01D92D3
:10071000A83CB207E1F713E0C2E7D3E004C0219799
:10072000FE010E94B139C137D107C9F70E94BF2726
:100730000C94053A0C940000E091FC03F0E0EE0FFD
:10074000FF1FE350FC4F808191810196918380834C
:100750008091E7029091E802A091E902B091EA024B
:100760000196A11DB11D8093E7029093E802A0932A
:10077000E902B093EA0281E08093280308958F9202
:100780009F92AF92BF92CF92DF92EF92FF920F9320
:100790001F93CF93DF93EC015A0149017A01C62ED2
:1007A000660FDD08C7018A199B0988159905B4F4FD
:1007B000A80160E070E0CE010E949533F7016193DB
:1007C0007F01B601CE010E94EA39009739F0FC01A1
:1007D0002081222319F0EC012196E4CFDF91CF9103
:1007E0001F910F91FF90EF90DF90CF90BF90AF904F
:1007F0009F908F900895CF93C82F10920A01109266
:1008000009011092690660E08EE596E00E945D0C99
:1008100010920601809107019091080197FD06C092
:100820008FEF9FEF9093080180930701CC2359F03D
:100830000E94F621809164068B7F80936406886015
:10084000CF910C94E521CF910895CF93DF93CEE51E
:10085000D6E08E81982F94609E838C600E94E52163
:1008600088E08B8760E0CE010E945D0C81E0809380
:10087000060180913E0190E090930A018093090166
:100880000E94F6218FEF9FEF90930801809307015C
:100890001092E6021092E502DF91CF9108954F92F7
:1008A0005F926F927F928F929F92AF92BF92CF9200
:1008B000DF92EF92FF92CF93C090D404D090D504F2
:1008C000E090D604F090D704C701B60120E831E5E6
:1008D00041E050E00E94F83749015A013093D304B7
:1008E0002093D20420E1422E2EE0522E612C712C56
:1008F000A30192010E94F8372093D104C701B601E9
:10090000A30192010E94F8373CE3432E512C612C45
:10091000712CA30192010E94F8372093D004C701E3
:10092000B601A30192010E94F8376093CF041092A0
:1009300006034AE065EC74E0C4010E94F93465ECFA
:1009400074E086E093E00E94DF3966E872E086E0BA
:1009500093E00E94DF39C091D104CA3018F067E6F5
:1009600072E002C062E872E086E093E00E94DF3944
:100970004AE065EC74E08C2F90E00E94F93465EC5D
:1009800074E086E093E00E94DF39C091D004CA3061
:1009900018F064E872E002C061E872E086E093E07B
:1009A0000E94DF394AE065EC74E08C2F90E00E94F1
:1009B000F93465EC74E086E093E00E94DF39C09181
:1009C000CF04CA3018F064E872E002C061E872E057
:1009D00086E093E00E94DF394AE065EC74E08C2FFA
:1009E00090E00E94F93465EC74E086E093E0CF91EA
:1009F000FF90EF90DF90CF90BF90AF909F908F903F
:100A00007F906F905F904F900C94DF39CF92DF9280
:100A1000EF92FF920F931F93CF93DF9300D000D0FC
:100A200000D0CDB7DEB78C0164E476E00E943A15C1
:100A30006BE376E0C8010E943A1540911B03509188
:100A40001C0360E070E02AE0C8010E94731568E3AF
:100A500076E0C8010E943A156FE276E0C8010E9474
:100A60003A154091EF025091F00260E070E02AE008
:100A7000C8010E9473156CE276E0C8010E943A1525
:100A800063E276E0C8010E943A154091EB02509172
:100A9000EC026091ED027091EE0222E030E0C801BC
:100AA0000E94161660E276E0C8010E943A1567E1DE
:100AB00076E0C8010E943A154091E7025091E802A1
:100AC0006091E9027091EA022AE0C8010E94731560
:100AD00064E176E0C8010E943A156BE076E0C80157
:100AE0000E943A154091D4045091D5046091D604E7
:100AF0007091D7042AE0C8010E94731566E076E081
:100B0000C8010E943A150E944F0469EF75E0C801C0
:100B10000E943A1568ED75E0C8010E943A1569EC2B
:100B200075E0C8010E943A1540910F0150E060E065
:100B300070E020E1C8010E9473154091100150E05F
:100B400060E070E020E1C8010E947315409111013E
:100B500050E060E070E020E1C8010E947315409110
:100B6000120150E060E070E020E1C8010E947315BE
:100B70004091130150E060E070E020E1C8010E9464
:100B800073154091140150E060E070E020E1C8016D
:100B90000E94731568EB75E0C8010E943A1566E083
:100BA00073E0C8010E94F81669EA75E0C8010E9466
:100BB0003A1540914001509141016091420170917C
:100BC000430122E030E0C8010E9416166AE975E090
:100BD000C8010E943A150E94A727BC01990F880BF3
:100BE000990B0E94B53620E030E048EC52E40E94B8
:100BF00014376B017C0180913F01682F70E080E029
:100C000090E00E94B5369B01AC01C701B6010E947D
:100C1000FF38AB01BC0121E030E0C8010E9416168C
:100C200060E975E0C8010E943A1540913F0150E02B
:100C300060E070E02AE0C8010E94731563E875E087
:100C4000C8010E943A1540913B0150913C0160E07F
:100C500070E02AE0C8010E94731566E775E0C801DC
:100C60000E943A1560913D0170E0C8010E94712711
:100C700067E675E0C8010E943A1540913E0150E0D8
:100C800060E070E02AE0C8010E94731568E575E035
:100C9000C8010E943A1560913A0170E0C8010E94B3
:100CA000712766E475E0C8010E943A1580913A0107
:100CB0009E012F5F3F4F7901882341F0C9010E94B7
:100CC0000E22B801C7010E94BC1505C062E475E0A0
:100CD000C8010E943A156FE275E0C8010E943A15FA
:100CE0004091150150E060E070E02AE0C8010E94E8
:100CF00073156DE275E0C8010E943A154091160126
:100D000050E060E070E02AE0C8010E9473156BE2D9
:100D100075E0C8010E943A154091170150E060E06B
:100D200070E02AE0C8010E94731569E275E0C8010D
:100D30000E943A154091180150E060E070E02AE00E
:100D4000C8010E9473156CE175E0C8010E943A1554
:100D500069E171E0C8010E94F81669E075E0C80118
:100D60000E943A158091C2069091C306009711F433
:100D700088EC96E0B701681B790BC8010E947127C7
:100D800069EE74E0C8010E943A1561E672E0C8019C
:100D90000E94F8166AED74E0C8010E943A1568E6F0
:100DA00072E0C8010E94F8166BEC74E0C8010E9462
:100DB0003A1564E772E0C8010E94F81662EC74E02C
:100DC000C8010E94021626960FB6F894DEBF0FBE29
:100DD000CDBFDF91CF911F910F91FF90EF90DF90EA
:100DE000CF900895CF93DF93EC01109275046EE8D5
:100DF00072E085E794E00E94DF394AE065EC74E038
:100E000080911B0390911C030E94F93480911A0376
:100E1000882339F04AE065EC74E080E090E00E94BD
:100E2000F93465EC74E085E794E00E94DF39BE0197
:100E300085E794E00E94DF3963E972E085E794E09A
:100E40000E94DF394AE065EC74E08091EF029091F6
:100E5000F0020E94F93465EC74E085E794E00E94AA
:100E6000DF39BE0185E794E00E94DF3968E972E06E
:100E700085E794E00E94DF394AE065EC74E08091F8
:100E8000E7029091E8020E94F93465EC74E085E78E
:100E900094E00E94DF39BE0185E794E00E94DF39CB
:100EA0006DE972E085E794E00E94DF396091EB0222
:100EB0007091EC028091ED029091EE020E947139E6
:100EC000DC01CB014AE065EC74E00E94F93465EC8A
:100ED00074E085E794E00E94DF39BE0185E794E085
:100EE0000E94DF3962EA72E085E794E00E94DF3910
:100EF0004AE065EC74E08091D4049091D5040E949E
:100F0000F93465EC74E085E794E00E94DF3985E709
:100F100094E0DF91CF91089510921C0310921B036F
:100F20001092EB021092EC021092ED021092EE027F
:100F30001092E7021092E8021092E9021092EA027F
:100F40001092F0021092EF0288E7EDEFF3E0DF017C
:100F50001D928A95E9F71092FC031092D404109226
:100F6000D5041092D6041092D70408951F920F92C0
:100F70000FB60F9211248F929F92AF92BF92CF9291
:100F8000DF92EF92FF922F933F934F935F936F9374
:100F90007F938F939F93AF93BF93CF93DF93EF9301
:100FA000FF93C090D404D090D504E090D604F09084
:100FB000D704C701B6016F5F7F4F8F4F9F4F60937C
:100FC000D4047093D5048093D6049093D704EDEFA6
:100FD000F3E0C0E0D0E021913191C20FD31F24E0B3
:100FE000E537F207C1F7D0931C03C0931B03209190
:100FF000EF023091F0022C173D0720F4D093F0025D
:10100000C093EF020E94B3362091EB023091EC02C4
:101010004091ED025091EE020E9414374B015C01A9
:10102000BE0180E090E00E94B3369B01AC01C50197
:10103000B4010E9493384B015C01C701B6016E5F99
:101040007F4F8F4F9F4F0E94B3369B01AC01C5016C
:10105000B4010E94FF386093EB027093EC0280931E
:10106000ED029093EE020E947139672B51F484E0F7
:101070000E94621761E0892B09F060E084E00E9421
:101080008B178091FC038F5F8093FC038C3328F0D7
:1010900081E0809326031092FC03E091FC03F0E0D2
:1010A000EE0FFF1FE350FC4F118210828091090167
:1010B00090910A01019790930A018093090181E0C0
:1010C00080930C01FF91EF91DF91CF91BF91AF9190
:1010D0009F918F917F916F915F914F913F912F9150
:1010E000FF90EF90DF90CF90BF90AF909F908F9048
:1010F0000F900FBE0F901F9018950F931F93CF93D3
:10110000DF9300D000D000D0CDB7DEB780913A0198
:10111000882309F48AC16EE973E087EA95E00E94AA
:101120003A158091F40381112AC01092DC031092C9
:10113000DB0388EE93E0A0E0B0E08093DD039093C2
:10114000DE03A093DF03B093E00389E891E090937E
:10115000DA038093D90381E592E09093E8038093CA
:10116000E7031092E9031092EA031092EB03109246
:10117000EC0384E08093F10381E08093F40386E93B
:1011800093E090935706809356066CE271E080E0FE
:1011900090E00E9479181FB7F8948091950381110F
:1011A00027C0E7ECF6E08491E9EAF6E09491E82FB5
:1011B000F0E0EE0FFF1FEF5AF94FA591B491EC91BB
:1011C000E92321F461E08AE00E948B1761E08AE064
:1011D0000E943D188CB580618CBD8CB580648CBD3F
:1011E00061E08DE00E943D1861E08BE00E943D18B7
:1011F000809195038F5F809395031FBF229A80E5AE
:1012000090E00E943E2660E880E090E00E94740D2D
:1012100065E58BE190E00E94740D65E58AE190E060
:101220000E94740D0E943D2680E090E49093980502
:101230008093970580E090E69093A00580939F05AA
:1012400080E098E490939A058093990580E098E671
:101250009093A2058093A10580E090E590939C0572
:1012600080939B0580E090E79093A4058093A3056D
:1012700080E098E590939E0580939D0580E098E737
:101280009093A6058093A50580E590E00E943E26F8
:1012900046E050E06FE071E089E090E00E94450D8B
:1012A00081E592E09A8389831B821C821D821E82C3
:1012B000CE0103960E9436260E943D268091560656
:1012C00090915706FC0112A213A214A215A216A215
:1012D00017A210A611A612A613A614A615A640E6DC
:1012E0005AEE60E070E046AB57AB60AF71AF40EADA
:1012F0005FE060E070E042AF53AF64AF75AFDC0118
:10130000189626E0FD01322F11923A95E9F7AC01CB
:10131000425F5F4F34E1FA0111923A95E9F7EFE04D
:10132000F1E001900D922A95E1F7FC01EE5BFF4F91
:1013300010820E9411208C018130910509F051C06A
:1013400080E590E00E943E26609156067091570617
:10135000625F7F4FCE0101960E94FA16CE0103967E
:101360000E94362660915606709157066A5E7F4F3E
:10137000CE0101960E94FA1644E050E0BE016D5F76
:101380007F4F81E090E00E94450D6091560670917C
:1013900057066E5E7F4FCE0101960E94FA1644E01A
:1013A00050E0BE016D5F7F4F85E090E00E94450DEB
:1013B0000E943D266091560670915706625E7F4FEF
:1013C000CE0101960E94FA168B819C81AD81BE816F
:1013D0008093520690935306A0935406B0935506FB
:1013E00009C0892B39F466E973E087EA95E00E9429
:1013F00002161DC0CE0101960E940E2267EA75E01A
:10140000CE0101960E94BC1565E672E087EA95E080
:101410000E945E1584E896E00E94FE1160E084E080
:101420000E948B1701E010E002C000E010E0C8014C
:1014300026960FB6F894DEBF0FBECDBFDF91CF91D9
:101440001F910F910895CF92DF92EF92FF920F9329
:101450001F93CF93DF93CDB7DEB72C970FB6F894D9
:10146000DEBF0FBECDBF9C878B87AE01455F5F4F50
:1014700060EA72E00E94D234BC01CE0101967C0188
:101480000E94FE396701F70101900020E9F73197CA
:10149000EE19FF09C6018E199F098E179F0758F490
:1014A000F6018081082E000C990B0E94C339F601C9
:1014B00081936F01E8CF19811F3319F463EC73E056
:1014C00030C1163469F48B859C850E94A7346093E3
:1014D000400170934101809342019093430145C1C3
:1014E000183439F48B859C850E94AB3480933F017E
:1014F0003CC1113449F48B859C850E94AB34909398
:101500003C0180933B0131C167EA72E0C7010E9450
:10151000F539892B39F40E948C07109285001092BE
:10152000840023C1123481F4EB85FC858181082E6F
:10153000000C990B0E94C33921E08E34910509F00B
:1015400020E020933D0111C1143549F48B859C8521
:101550000E94AB34893708F406C188E704C11C3403
:1015600091F4EB85FC858181082E000C990B0E947B
:10157000C3398E34910519F40E942504F6C081E028
:101580000E94FB03F2C01E34E9F4EB85FC858181E7
:10159000082E000C990B0E94C33921E08E3491056E
:1015A00009F020E020933A01222349F00E947D08AF
:1015B00021E0892B09F420E020932703D6C0109264
:1015C0002703D3C06DEA72E0C7010E94F539892B69
:1015D000A1F48B859C85FC0101900020E9F79F0117
:1015E000225131092817390741F400E110E026E0C3
:1015F00030E04FE051E06AE315C01335B1F48B855C
:101600009C85FC0101900020E9F79F0120513109E0
:101610002817390751F40AE010E024E030E045E1F2
:1016200051E06EE20E94BF03A0C061EB72E0C7010F
:101630000E94F539892B39F46B857C8589E191E02D
:101640000E94FE3992C01D34C9F58A818534E9F5BE
:1016500066EB73E087EA95E00E943A156E01F9E0C7
:10166000CF0ED11C8091C2069091C306009711F451
:1016700088EC96E0C81AD90A0D2C000CEE08FF0879
:10168000F7FE0EC06DE287EA95E00E94331544270D
:101690005527BA014C195D096E097F092AE003C07C
:1016A0002AE0B701A60187EA95E00E94731565E676
:1016B00072E087EA95E00E945E1557C01F3429F456
:1016C00087EA95E00E94060550C065EB72E0C7010D
:1016D0000E94F539892B19F40E94BC2146C01635A9
:1016E00029F561E672E087EA95E00E94F81663EB5F
:1016F00073E087EA95E00E943A1568E672E087EAAF
:1017000095E00E94F8166091F10287EA95E00E9448
:10171000331564E772E087EA95E00E94F81660EB03
:1017200073E087EA95E00E9402161FC06CEB72E03E
:10173000C7010E94F539892B21F481E080932503AC
:1017400014C061EC72E087EA95E00E945E1565E6E0
:1017500072E087EA95E00E945E1587EA95E00E94B4
:101760009D1480E007C080933E0187EA95E00E94C7
:101770009D1481E02C960FB6F894DEBF0FBECDBF4E
:10178000DF91CF911F910F91FF90EF90DF90CF905D
:1017900008959091E4028091E302981750F4E92FA4
:1017A000F0E0E450FB4F208130E09F5F9093E40233
:1017B00002C02FEF3FEFC90108958091E30290E04E
:1017C0002091E402821B910908950895CF92DF923F
:1017D000EF92FF920F931F93CF93DF937C01262FFD
:1017E000972F8A018091FB04882391F0C62FD72F71
:1017F0006E01C40ED51ECC15DD0571F06991D701BF
:10180000ED91FC910190F081E02DC7010995F3CF96
:10181000642F822F0E94851AC801DF91CF911F91FA
:101820000F91FF90EF90DF90CF900895CF93DF93CB
:101830001F92CDB7DEB769832091FB042223D1F03C
:101840002091E102203240F021E030E0FC013383BE
:10185000228380E090E015C08091E202E82FF0E062
:10186000E552FB4F998190838F5F8093E2028093D2
:10187000E10205C061E0CE0101960E94851A81E077
:1018800090E00F90DF91CF9108951F93CF93DF9356
:10189000182F66E270E00E944711C82FD0E067E27F
:1018A00070E0812F0E944711DC2FCC279E01282B4E
:1018B000C901DF91CF911F910895CF93FC01C4819D
:1018C00021E02093FB04C093DA041092E20210920C
:1018D000E1028385682B84E496E00E94160C8091D7
:1018E000E102813208F046C09091E0029111FCCFF4
:1018F00092E09093E00291E09093DF029FEF90934B
:101900001C0510923E0580933D05ABEDB4E02DE142
:1019100035E0F9019E2F921B981718F49D91919331
:10192000F9CF10923F0580913F05CC0FC82BC09393
:101930003F058091DE02813061F41092DE028091D9
:101940003F058093BB008091BC0083FDF8CF85EC00
:1019500001C085EE8093BC008091E0028230E1F30B
:1019600080911C058F3F31F080911C05803211F071
:1019700080911C051092E2021092E1021092FB0489
:10198000CF9108950F931F93CF938C01C62F0E9480
:101990005D0C6C2F6460C8010E945D0C6C2F6B7F26
:1019A000C8010E945D0C83EC90E00197F1F7CF91A4
:1019B0001F910F9108950F931F93CF938C01C62F02
:1019C000607F61600E94C20C80E1C89FB001112459
:1019D0006160C8010E94C20C81E090E0CF911F912C
:1019E0000F9108952A9A08952A9808951F93CF93E6
:1019F000DF93182F60E270E00E944711C82FD0E0FB
:101A000061E270E0812F0E944711DC2FCC279E01FC
:101A1000282BC901DF91CF911F9108958EBD000041
:101A20000DB407FEFDCF8EB50895CF92DF92EF92F1
:101A3000FF920F931F93CF93DF93EC017A018B01F9
:101A40006C01C40ED51ECC15DD05A9F00E94F40C66
:101A50008FE00E940E0D8D2F0E940E0D8C2F0E9484
:101A60000E0D219680E00E940E0DF80181938F01EA
:101A70000E94F20CE8CFC701DF91CF911F910F9127
:101A8000FF90EF90DF90CF900895CF92DF92EF928A
:101A9000FF920F931F93CF93DF93EC017A018B0199
:101AA0006C01C40ED51ECC15DD05A1F00E94F40C0E
:101AB00080EF0E940E0D8D2F0E940E0D8C2F0E9424
:101AC0000E0D2196F80181918F010E940E0D0E944A
:101AD000F20CE9CFC701DF91CF911F910F91FF90D9
:101AE000EF90DF90CF9008951F93CF93DF9300D0B6
:101AF000CDB7DEB7182F6A8399830E94F40C80EF6C
:101B00000E940E0D9981892F0E940E0D812F0E9437
:101B10000E0D6A81862F0E940E0D0E94F20C81E04C
:101B20000F900F90DF91CF911F9108951F93CF9346
:101B3000DF9300D0CDB7DEB7182F80E590E0698342
:101B40007A830E943E2621E041E050E069817A815B
:101B5000812F0E942C220E943D2681E090E00F9070
:101B60000F90DF91CF911F910895CF93DF931F9234
:101B7000CDB7DEB7FC01218D328D232B49F0BE019C
:101B80006F5F7F4F808D0E94960D898190E002C02B
:101B90008FEF9FEF0F90DF91CF910895FF920F93FA
:101BA0001F93CF93DF93F82E80E590E00E943E26AE
:101BB000C0E0D0E08F2D0E94450C8C01892B21F0D4
:101BC0008F2D0E94450CEC01C017D10799F70E9498
:101BD0003D26CE01DF91CF911F910F91FF90089587
:101BE000AF92BF92CF92DF92EF92FF921F93CF936B
:101BF000DF93182F5B017A0180E590E00E943E267A
:101C0000C0E0D0E0812F0E94450C6C01892B21F0AF
:101C1000812F0E94450CEC01CC15DD0599F720972A
:101C200099F463E070E0812F0E9447118431F1F054
:101C30008823E1F0C1E0D0E08C3111F4C0E0D0E0C5
:101C4000D195C195D10912C0EC16FD060CF4E7013F
:101C50001C161D065CF420E0AE01B501812F0E9428
:101C60002C2260E470E0812F0E94FE210E943D261C
:101C7000CE01DF91CF911F91FF90EF90DF90CF9039
:101C8000BF90AF900895CF93DF93FC01218D328DEB
:101C90002115310519F48FEF9FEF11C0EC014217A8
:101CA000530708F0A901888D0E94F00D1816190637
:101CB00094F7298D3A8D281B390B3A8F298FDF91A4
:101CC000CF9108950F931F93CF93DF931F92CDB7BA
:101CD000DEB7FC01218D328D232B61F08C0141E0B8
:101CE00050E0BE016F5F7F4F808D0E94F00D18168F
:101CF00019061CF08FEF9FEF08C0F801818D928DBF
:101D00000197928F818F898190E00F90DF91CF9121
:101D10001F910F9108950F931F93CF93DF93CDB72A
:101D2000DEB728970FB6F894DEBF0FBECDBF8C018B
:101D3000F801818D928D892B49F0D801ED91FC91AC
:101D40000284F385E02DC8010995F2CF808D0E94B1
:101D5000CE0D181619065CF548E050E0BE016F5F25
:101D60007F4FD80158968C910E94F00D9C01181657
:101D70001906DCF489819A81AB81BC81F801808BE2
:101D8000918BA28BB38B8D8190E0982F88272E8129
:101D9000820F911D958B848B2F8130E0322F22276B
:101DA0008885280F311D328F218FC90102C080E044
:101DB00090E028960FB6F894DEBF0FBECDBFDF913E
:101DC000CF911F910F910895CF93C82F80E590E098
:101DD0000E943E2660E170E08C2F0E94FE214FEFB2
:101DE00062E070E08C2F0E943D11CF910C943D2653
:101DF000FF920F931F93CF93DF9300D0CDB7DEB741
:101E0000F82E8A012A8369830E94E40E80E590E01F
:101E10000E943E262A816981462F422B60E070E0B5
:101E20008F2D0E943D110115110551F40091D80428
:101E30001091D9040F5F1F4F1093D9040093D80459
:101E4000412F64E070E08F2D0E943D11402F65E02E
:101E500070E08F2D0E943D1161E070E08F2D0E9497
:101E6000FE210E943D2681E00F900F90DF91CF91DF
:101E70001F910F91FF900895BF92CF92DF92EF9242
:101E8000FF920F931F93CF93DF9300D000D000D029
:101E9000CDB7DEB7FC01208D243009F053C06A01B4
:101EA0007B018C01B12C63E070E08B2D0E94471107
:101EB000811103C0F801B08E06C08831D9F3B39404
:101EC000F4E0BF12F0CFF801808D8430D9F196E0B4
:101ED000E7E5F1E0DE01119601900D929A95E1F7A8
:101EE000F70193819F779C8394819D8395819E8345
:101EF000B7016E5F7F4F90E0982F882744E050E055
:101F0000845F9B4F0E94450DB601F801808D0E94B1
:101F1000A511F801808D90E0982F882746E050E0C9
:101F2000BE016F5F7F4F8A5F9B4F0E94450DF80196
:101F3000128E118E20E8A60162E0808D0E94F80EBC
:101F400081E001C080E026960FB6F894DEBF0FBE98
:101F5000CDBFDF91CF911F910F91FF90EF90DF9058
:101F6000CF90BF9008951F93CF93DF931F92CDB76B
:101F7000DEB7182F80E590E00E943E2663E070E017
:101F8000812F0E94471189830E943D2689810F90ED
:101F9000DF91CF911F910895CF93DF931F92CDB71B
:101FA000DEB76983DC01ED91FC910280F381E02DC5
:101FB00041E050E0BE016F5F7F4F09950F90DF91C8
:101FC000CF910895FC01818D928D0895FC01848943
:101FD0009589089521E532E0FC0131832083FB01DE
:101FE0004089518962897389FC01428353836483E8
:101FF00075830895DC01ED91FC91048CF58DE02D45
:10200000099480E00895CF93DF931F92CDB7DEB798
:102010006983DC01ED91FC910280F381E02D41E0C8
:1020200050E0BE016F5F7F4F09950F90DF91CF9118
:102030000895FC019485FB018485981303C081E019
:10204000943009F480E0089521E0FC018485843017
:1020500009F420E0822F08950895AF92BF92CF92A5
:10206000DF92FF920F931F93CF93DF938C015B015D
:10207000EA01FC01C688D788F08C80E590E00E94D8
:102080003E268F2D0E94F9228C179D0720F48F2D5C
:102090000E94F922EC019E01A501B6018F2D0E943C
:1020A00094220E943D26F801868997898C0F9D1FF6
:1020B000978B868BCE01DF91CF911F910F91FF906F
:1020C000DF90CF90BF90AF900895CF92DF92EF92C4
:1020D000FF920F931F93CF93DF93CDB7DEB7AF97E8
:1020E0000FB6F894DEBF0FBECDBF7C016A0101E5DB
:1020F00012E01A8309831C861B8688EE93E0A0E019
:10210000B0E08D879E87AF87B88B89E891E09A878A
:102110008987188F0F8B198E1A8E1B8E1C8E84E068
:1021200089A31DA30CA31EA21FA218A619A6809105
:10213000520690915306A0915406B09155068CA773
:102140009DA7AEA7BFA78B839C83AD83BE83188654
:102150001F82AE014C5D5F4FCE0101960E94961D1D
:1021600081309105B1F4D701ED91FC910488F58996
:10217000E02D1BA70AA78EA19FA1A8A5B9A58CA792
:102180009DA7AEA7BFA7A601BE01665D7F4FC70191
:102190000995AF960FB6F894DEBF0FBECDBFDF91A5
:1021A000CF911F910F91FF90EF90DF90CF90089506
:1021B000CF93DF93EC01888D843061F00E94E40EB0
:1021C000E88DF0E0EE0FFF1FE35EFC4F11821082FE
:1021D00084E0888FDF91CF910895EF92FF921F9353
:1021E000CF93DF93FC01208D243011F080E01CC0E0
:1021F0007B01EC0110E0812F0E94B30F811102C01E
:10220000188F05C08831E1F31F5F1430A1F7888D66
:10221000843061F3FD86EC861A8E198E20E0A701CA
:1022200062E00E94F80E81E0DF91CF911F91FF9054
:10223000EF9008950F931F93CF93DF931F92CDB725
:10224000DEB78C01DC01ED91FC910084F185E02D7D
:102250000995892B51F0BE016F5F7F4FF80184858E
:102260000E94960D898190E002C08FEF9FEF0F9042
:10227000DF91CF911F910F9108959B0190E00496FB
:10228000982F8827642F820F931F0C94740D0F933F
:102290001F93CF93DF931F92CDB7DEB790E00496E4
:1022A000982F88278C01060F171F0E94F40C8FE0CF
:1022B0000E940E0D812F0E940E0D802F0E940E0D88
:1022C00080E00E940E0D89830E94F20C89810F909C
:1022D000DF91CF911F910F910895CF93FC01C08D95
:1022E00080E590E00E943E2660E270E08C2F0E9424
:1022F000FE2162E070E08C2F0E94471184FD19C01E
:1023000062E070E08C2F0E94471183FF0BC048E110
:1023100062E070E08C2F0E943D110E943D2680E01B
:1023200090E011C00E943D2680E590E00E943E268C
:10233000E0CF40E162E070E08C2F0E943D110E94EE
:102340003D2681E090E0CF910895CF93DF93C82F91
:10235000D62F472F60E170E00E943D114D2F61E1C3
:1023600070E08C2FDF91CF910C943D11FF920F9371
:102370001F93CF93DF93FB01DC0157961C921E92B3
:1023800056975896FC908281811109C083818111F2
:1023900006C08481811103C085818823F9F041152D
:1023A0005105E1F08A01EF0180E590E00E943E26B0
:1023B000BE016E5F7F4F2F2D30E0922F882744E0C3
:1023C00050E0845F9B4F0E94450DB8018F2D0E9405
:1023D000A5110E943D2681E090E002C080E090E0DF
:1023E000DF91CF911F910F91FF900895FC0184859B
:1023F000843011F00C94B30F80E008958F929F9277
:10240000AF92BF92CF92DF92EF92FF920F931F9302
:10241000CF93DF93CDB7DEB72D970FB6F894DEBF1D
:102420000FBECDBF7C0100E010E038EE832E33E01C
:10243000932EA12CB12C41E1C42E42E0D42E1C825B
:102440001B828D829E82AF82B886DA82C9820D8716
:10245000CE0101960E94F611811125C0F701448139
:10246000558120E061E0802F0E94F80E80E590E029
:102470000E943E2663E070E0802F0E944711833166
:1024800029F462E070E0802F0E94FE210E943D2628
:10249000F70184819581000F111FF801E35EFC4F65
:1024A0009183808305C00F5F1F4F0430110539F6FB
:1024B0002D960FB6F894DEBF0FBECDBFDF91CF9142
:1024C0001F910F91FF90EF90DF90CF90BF90AF9052
:1024D0009F908F900895CF93DF93FC012485243043
:1024E000D1F0EC010E94F611843181F0882371F063
:1024F000883161F08C3161F4E881F9810084F185E3
:10250000E02DCE01099521E0892B19F420E001C0CE
:1025100021E0822F01C080E0DF91CF910895CF921A
:10252000DF92EF92FF921F93CF93DF93FC0114850C
:102530001430A9F1EC0180E590E00E943E2668E0AD
:1025400070E0812F0E94FE210E943D260E94B31858
:102550006B017C01CE010E94F6118823B1F061E08D
:1025600070E080E090E00E9479180E94B318DC01CE
:10257000CB018C199D09AE09BF09883E9340A10586
:10258000B10540F38C850E94E40EEC85F0E0EE0F7F
:10259000FF1FE35EFC4F1182108284E08C87DF9185
:1025A000CF911F91FF90EF90DF90CF9008954F92C1
:1025B0005F926F927F928F929F92AF92BF92CF92D3
:1025C000DF92EF92FF921F93CF93DF93CDB7DEB7E9
:1025D0002D970FB6F894DEBF0FBECDBF7C019DE1F5
:1025E000A92E93E0B92E10E0C12CD12C28EE422E5A
:1025F00023E0522E612C712C31E1832E32E0932E98
:102600001C821B824D825E826F8278869A828982CA
:102610001D87D5012D913D915D01F7018481958143
:1026200028173907B1F4CE0101960E94F6118431C2
:1026300069F0CE0101960E94F6118C3151F4CE0161
:1026400001960E94BA25892B91F003C0CC24C39433
:10265000D12C1F5F1430A1F6CD2871F4D701ED9174
:10266000FC910084F185E02DC701099505C0CE01DC
:1026700001960E948F12EDCF2D960FB6F894DEBF13
:102680000FBECDBFDF91CF911F91FF90EF90DF90F4
:10269000CF90BF90AF909F908F907F906F905F9002
:1026A0004F9008952F923F924F925F926F927F9238
:1026B0008F929F92AF92BF92CF92DF92EF92FF9252
:1026C0000F931F93CF93DF93CDB7DEB72E970FB63F
:1026D000F894DEBF0FBECDBF7C016B015A010E9492
:1026E000D7120DE113E020E0612C712C88EE282E2A
:1026F00083E0382E412C512C91E1892E92E0992EC5
:102700001C821B822D823E824F8258869A82898249
:102710002D87F801419151918F01F70184819581B5
:102720004817590741F4CE0101962E870E94F611F1
:102730002E858731E9F02F5F243011F7C3012E96E3
:102740000FB6F894DEBF0FBECDBFDF91CF911F91C2
:102750000F91FF90EF90DF90CF90BF90AF909F9040
:102760008F907F906F905F904F903F902F90089543
:10277000A501B601CE0101962E870E944126680E62
:10278000791E2E85D8CFCF92DF92EF92FF920F93D2
:102790001F93CF93DF936C017A018B01C0E0D0E0EF
:1027A000CE15DF0589F0D8016D918D01D601ED912F
:1027B000FC910190F081E02DC6010995892B11F45F
:1027C0007E0102C02196ECCFC701DF91CF911F910E
:1027D0000F91FF90EF90DF90CF900895FC01538D03
:1027E000448D252F30E0842F90E0821B930B5417EB
:1027F00010F0CF96089501970895FC01918D828D78
:10280000981761F0828DDF01A80FB11D5D968C9144
:10281000928D9F5F9F73928F90E008958FEF9FEF4F
:102820000895FC01918D828D981731F0828DE80F0B
:10283000F11D858D90E008958FEF9FEF0895FC01C5
:10284000918D228D892F90E0805C9F4F821B910992
:102850008F739927089587EA95E00E941F1421E05D
:10286000892B09F420E0822F0895FC01848DDF017B
:10287000A80FB11DA35ABF4F2C91848D90E00196F3
:102880008F739927848FA689B7892C93A089B189E2
:102890008C9180648C93938D848D981306C00288EC
:1028A000F389E02D80818F7D80830895EF92FF92E0
:1028B0000F931F93CF93DF93EC0181E0888F9B8D63
:1028C0008C8D981305C0E889F989808185FD24C025
:1028D000F62E0B8D10E00F5F1F4F0F731127E02EA8
:1028E0008C8DE8120CC00FB607FCFACFE889F98985
:1028F000808185FFF5CFCE010E943514F1CF8B8DFD
:10290000FE01E80FF11DE35AFF4FF0820B8FEA89B9
:10291000FB898081806207C0EE89FF896083E88936
:10292000F98980818064808381E090E0DF91CF919C
:102930001F910F91FF90EF900895CF93DF93EC01DB
:10294000888D8823C9F0EA89FB89808185FD05C0CF
:10295000A889B9898C9186FD0FC00FB607FCF5CF09
:10296000808185FFF2CFA889B9898C9185FFEDCF51
:10297000CE010E943514E7CFDF91CF91089580E01A
:1029800090E0892B29F00E942B1481110C940000F7
:102990000895833081F028F4813099F08230A1F0DD
:1029A00008958730A9F08830B9F08430D1F480914F
:1029B00080008F7D03C0809180008F77809380009E
:1029C000089584B58F7702C084B58F7D84BD089546
:1029D0008091B0008F7703C08091B0008F7D80938D
:1029E000B00008953FB7F89480918C0590918D05C3
:1029F000A0918E05B0918F0526B5A89B05C02F3FED
:102A000019F00196A11DB11D3FBFBA2FA92F982F14
:102A10008827820F911DA11DB11DBC01CD0142E08F
:102A2000660F771F881F991F4A95D1F7089508955B
:102A300085ED8093BC008091BC0084FDFCCF10929A
:102A4000E0020895089581E090E03091E402209141
:102A5000E302321710F480E090E09195819591099E
:102A600008950E94BE39DC01ED91FC910190F08146
:102A7000E02D0994EF92FF920F931F93CF93DF9372
:102A80008C017B01C0E0D0E0F701EC0FFD1F6491E9
:102A9000662361F0D801ED91FC910190F081E02D69
:102AA000C8010995892B11F02196EECFCE01DF9157
:102AB000CF911F910F91FF90EF90089561157105CF
:102AC00079F0FB0101900020E9F73197AF01461B37
:102AD000570BDC01ED91FC910280F381E02D09940C
:102AE00080E090E008954F925F926F927F92EF9214
:102AF000FF920F931F93CF93DF93CDB7DEB7A197CC
:102B00000FB6F894DEBF0FBECDBF7C01FA01CB013A
:102B100019A2223008F42AE08E010F5D1F4F422EC9
:102B2000512C612C712CBF01A30192010E94F83736
:102B3000F901CA01015011096A3014F4605D01C045
:102B4000695CD8016C93232B242B252B61F7B801EA
:102B5000C7010E945E15A1960FB6F894DEBF0FBEA6
:102B6000CDBFDF91CF911F910F91FF90EF907F909C
:102B70006F905F904F9008958F929F92AF92BF9207
:102B8000CF92DF92EF92FF920F931F93CF93DF9339
:102B90007C018B016C0182E0C80ED11C4701E5E08D
:102BA0008E0E911CC0E0D0E0F60141916F0150E023
:102BB00060E070E02AE0C8010E9473155C016EE2DB
:102BC000C8010E9433158A0D9B1DC80FD91FC81458
:102BD000D90451F7F701458150E060E070E02AE048
:102BE000C8010E9473158C0F9D1FDF91CF911F911B
:102BF0000F91FF90EF90DF90CF90BF90AF909F909C
:102C00008F9008950F931F93CF93DF93EC010E9451
:102C10003A158C0165E672E0CE010E945E15800FC8
:102C2000911FDF91CF911F910F9108954F925F9265
:102C30006F927F928F929F92AF92BF92CF92DF92CC
:102C4000EF92FF92CF93DF93EC016A017B01B22EEA
:102C50009A01AB01C701B6010E94AC39882319F073
:102C60006AEC72E027C026013701E89477F82FEF6D
:102C70003FEF4FE75FE7C301B2010E94AC3981111A
:102C80000DC02FEF3FEF4FE75FE7C301B2010E9496
:102C9000AE3618161CF46EEC72E00CC02FEF3FEF4E
:102CA0004FE75FE4C701B6010E94A73918169CF4EC
:102CB00062ED72E0CE01DF91CF91FF90EF90DF9057
:102CC000CF90BF90AF909F908F907F906F905F90CC
:102CD0004F900C945E152FEF3FEF4FE75FECC7016D
:102CE000B6010E94AE3687FDE3CF20E030E0A901B7
:102CF000C701B6010E94AE3687FF0AC06DE2CE0161
:102D00000E9433154C01F7FAF094F7F8F09402C0E2
:102D1000812C912CA12C60E070E080E09FE3AB144B
:102D200040F420E030E040E251E40E94FF38A394F8
:102D3000F6CF9B01AC01C701B6010E9493382B016D
:102D40003C010E9478396B017C010E94B3369B01E3
:102D5000AC01C301B2010E9492382B013C012AE070
:102D6000B701A601CE010E9473157C01E80CF91C85
:102D7000BB2031F06EE2CE010E943315E80EF91E41
:102D8000DB2CDD2029F120E030E040E251E4C301FA
:102D9000B2010E9414372B013C010E9478394B018B
:102DA000A12CB12C2AE0B501A401CE010E9473151B
:102DB000E80EF91EC501B4010E94B3369B01AC01B7
:102DC000C301B2010E9492382B013C01DA94D9CFA1
:102DD000C701DF91CF91FF90EF90DF90CF90BF9030
:102DE000AF909F908F907F906F905F904F900895DD
:102DF0000C945E1521E532E0FC0131832083FB0158
:102E00004081518162817381FC01428353836483D9
:102E1000758308951F920F920FB60F9211242F936E
:102E20003F934F935F936F937F938F939F93AF9352
:102E3000BF93EF93FF9387EA95E00E943514FF91CB
:102E4000EF91BF91AF919F918F917F916F915F9122
:102E50004F913F912F910F900FBE0F901F9018959B
:102E60001F920F920FB60F9211242F938F939F935F
:102E7000EF93FF93E091B705F091B8058081E09161
:102E8000BD05F091BE0582FD12C090818091C00504
:102E90008F5F8F732091C105821751F0E091C005BB
:102EA000F0E0E955FA4F958F8093C00501C080810D
:102EB000FF91EF919F918F912F910F900FBE0F90E7
:102EC0001F901895CF93DF93282F30E0F901EB592D
:102ED000F94F8491F901E156F94FD491F901E35486
:102EE000F94FC491CC2391F081110E94C914EC2FA9
:102EF000F0E0EE0FFF1FE55AF94FA591B491EC9168
:102F0000ED2381E090E021F480E002C080E090E0D9
:102F1000DF91CF9108951F93CF93DF93282F30E057
:102F2000F901EB59F94F8491F901E156F94FD49128
:102F3000F901E354F94FC491CC23C9F0162F811144
:102F40000E94C914EC2FF0E0EE0FFF1FED54F94F73
:102F5000A591B4918FB7F894111105C09C91ED2FF4
:102F6000E095E92302C0EC91ED2BEC938FBFDF914C
:102F7000CF911F9108951F920F920FB60F921124B7
:102F80002F933F934F935F936F937F938F939F9371
:102F9000AF93BF93EF93FF93809193059091940526
:102FA000A0919505B0919605892B8A2B8B2B59F111
:102FB00080919005E0919105F0919205908189278B
:102FC00080838091930590919405A0919505B0918F
:102FD0009605181619061A061B060CF03DC08091BE
:102FE000930590919405A0919505B0919605019750
:102FF000A109B1098093930590939405A093950539
:10300000B093960529C080910D01E1EDF6E0E491C1
:103010009FEF90930D01E130B9F098F0E230C9F4E0
:10302000909170009D7F9093700091E09093B0001C
:103030009091B100987F94609093B1001092B3008A
:1030400008C010926E0005C090916F009D7F909314
:103050006F0060E00E948B17FF91EF91BF91AF91DD
:103060009F918F917F916F915F914F913F912F91A0
:103070000F900FBE0F901F901895CF93DF9390E0A5
:10308000FC01E156F94F2491FC01E354F94F84917E
:10309000882361F190E0880F991FFC01EF5AF94FE6
:1030A000C591D491FC01ED54F94FA591B4916111F2
:1030B00009C09FB7F8948881209582238883EC917A
:1030C0002E230BC0623061F49FB7F8943881822FB1
:1030D000809583238883EC912E2B2C939FBF06C071
:1030E0008FB7F894E8812E2B28838FBFDF91CF9183
:1030F00008958F929F92AF92BF92CF92DF92EF92FC
:10310000FF926B017C010E94F2144B015C01C1141F
:10311000D104E104F104F1F00E94F214DC01CB01CE
:1031200088199909AA09BB09883E9340A105B105F0
:1031300070F321E0C21AD108E108F10888EE880E88
:1031400083E0981EA11CB11CC114D104E104F10458
:1031500019F7DDCFFF90EF90DF90CF90BF90AF9049
:103160009F908F9008952FB7F89460918805709183
:10317000890580918A0590918B052FBF08951F9234
:103180000F920FB60F9211242F933F938F939F931B
:10319000AF93BF938091880590918905A0918A058E
:1031A000B0918B053091870523E0230F2D3720F454
:1031B0000196A11DB11D05C026E8230F0296A11D91
:1031C000B11D209387058093880590938905A0936E
:1031D0008A05B0938B0580918C0590918D05A09107
:1031E0008E05B0918F050196A11DB11D80938C05B0
:1031F00090938D05A0938E05B0938F05BF91AF91ED
:103200009F918F913F912F910F900FBE0F901F9024
:1032100018951F920F920FB60F9211242F933F9380
:103220004F935F936F937F938F939F93AF93BF93CE
:10323000EF93FF93E0910401F09105010995FF914F
:10324000EF91BF91AF919F918F917F916F915F911E
:103250004F913F912F910F900FBE0F901F90189597
:103260001F920F920FB60F9211242F933F934F93FB
:103270005F936F937F938F939F93AF93BF93EF93DE
:10328000FF93E0910201F09103010995FF91EF9105
:10329000BF91AF919F918F917F916F915F914F916E
:1032A0003F912F910F900FBE0F901F9018951F9276
:1032B0000F920FB60F9211242F933F934F935F936A
:1032C0006F937F938F939F93AF93BF93EF93FF93EE
:1032D0008091B900887F803609F49CC068F58832F7
:1032E00009F45BC090F4803109F454C038F48823A9
:1032F00009F4F6C0883009F44DC0F6C0883109F4ED
:103300004CC0803209F45DC0EFC0803409F468C05D
:1033100048F4803309F455C0883309F0E5C0809340
:103320001C05D8C0803509F44FC0883509F45DC04C
:10333000883409F0D9C0D6C0883909F4C7C0A8F4C8
:10334000883709F467C038F4883609F463C08037D9
:1033500009F460C0C9C0883809F4B8C0803909F4DC
:103360005FC0803809F0C0C05BC0803B09F486C0F4
:1033700038F4803A09F466C0883A09F47FC0B4C0D2
:10338000803C09F4A7C0883C09F4A4C0883B09F438
:103390008AC0AAC080913F0510C090913E058091DF
:1033A0003D05981770F5E0913E0581E08E0F809302
:1033B0003E05F0E0E35EFA4F80818093BB0085EC30
:1033C00086C080931C058EC0E0913E0581E08E0F83
:1033D00080933E058091BB00F0E0E35EFA4F80836E
:1033E00090913E0580913D056EC0E0913E0581E0E3
:1033F0008E0F80933E058091BB00F0E0E35EFA4FB4
:1034000080838091DF0281116DC081E08093DE02B4
:1034100084EA61C083E08093E00210928605CFCFFA
:1034200080918605803208F051C0E091860581E0E8
:103430008E0F809386058091BB00F0E0EA59FA4F29
:103440008083BDCF85EC8093BC001092E002809118
:103450008605803230F4E0918605F0E0EA59FA4FB3
:1034600010826091860570E0E0916405F091650539
:1034700086E695E009951092860536C084E0809333
:10348000E0021092630510926205E0916005F091F0
:103490006105099580916205811105C081E08093E5
:1034A000620510924005E091630581E08E0F8093E4
:1034B0006305F0E0E05CFA4F80818093BB0090915F
:1034C000630580916205981708F479CF85E88093A9
:1034D000BC000AC085EC8093BC001092E00204C0DE
:1034E00010921C050E941815FF91EF91BF91AF91AA
:1034F0009F918F917F916F915F914F913F912F910C
:103500000F900FBE0F901F90189540916205262FC7
:1035100030E0240F311D21323105DCF42091E0022E
:103520002430C9F4FC0180E090E0861758F4309113
:1035300062052191DC01A05CBA4FA30FB11D2C9351
:103540000196F3CF80916205680F6093620580E079
:10355000089581E0089582E0089580E3FB0180836F
:103560003296842F82958F7090E1899F40191124A3
:103570004A3014F4405D01C0495C4293482F8111E8
:10358000F0CF08952F923F924F925F926F927F9269
:103590008F929F92AF92BF92CF92DF92EF92FF9263
:1035A0000F931F93CF93DF93CDB7DEB7E3970FB69B
:1035B000F894DEBF0FBECDBF7C011A012B0139018B
:1035C0000E94B3184B015C0187010D5B1F4FC801BE
:1035D0000E948B0E18161906A4F00E94B318DC0185
:1035E000CB0188199909AA09BB09281639064A0688
:1035F0005B06D8F062E370E080E090E00E9479180A
:10360000E6CF42E250E0BE016F5F7F4FC8010E94EB
:10361000430E8981823011F080E061C1F801848914
:10362000958983349105C1F702C08FEF58C16D8130
:103630007E818F8198850E94B7394B015C01F3012F
:10364000608371838283938346E050E0B701685FB3
:103650007F4FCE014D960E94CB39892BE9F6F701B9
:1036600080819181A281B38188169906AA06BB0642
:1036700098F284819581A681B78188159905AA055C
:10368000BB0550F289899A89AB89BC89868797875F
:10369000A08BB18B8EECA82EB12CC8010E94620EBB
:1036A000F1E0AF1AB108C9F719A6670182E2C80EA6
:1036B000D11CF701B696FBA7EAA7C7018A969DA77A
:1036C0008CA73C974F0189969FA78EA73897F9AB97
:1036D000E8AB1701F6E12F0E311CC5979BAB8AAB07
:1036E000F801818D928D181619060CF0F7C0C801EB
:1036F0000E94620E8333910509F4CBC0FCF4813043
:103700009105C9F11CF4892B59F3DCC08330910574
:10371000D1F1069709F0D6C0C8010E94620E5C0183
:1037200044E050E06AA97BA9C8010E94430E412CE5
:10373000512CBB24F4E0AF1AB10840C08A33910584
:1037400009F47BC03CF48533910569F0C69709F410
:1037500040C0B8C08B33910509F485C08F3F9105F7
:1037600009F4BECFAFC0C8010E94620EC8010E941A
:10377000620E89A7B5CFC8010E94620E44E050E0F6
:1037800068A979A93AC0C8010E94620E5C0144E0B0
:1037900050E0B101C8010E94430E412C512CBB24C2
:1037A00094E0A91AB1084A145B040CF099CFC8013F
:1037B0000E94620EEFEF4E1A5E0AF5CF4A145B04C8
:1037C0000CF08ECFC8010E94620E8FEF481A580A83
:1037D000F5CFC8010E94620EB82EF701828D8111CB
:1037E00010C0838D81110DC0848D81110AC0858D1B
:1037F000811107C044E050E0B401C8010E94430EAB
:103800006FCFEEA5FFA54080518062807380B40128
:10381000CE0183960E94FA168DA19EA1AFA1B8A5F4
:1038200084159505A605B70529F3BB2009F458CFE3
:10383000C8010E94620EBA94F8CFC8010E94620EBD
:1038400044E050E06AA57BA5C8010E94430EF70141
:1038500066A177A180A591A50E94B73966A377A339
:1038600080A791A73DCFC8010E94620E44E050E0BE
:103870006CA57DA5C8010E94430EF70162A573A542
:1038800084A595A50E94B73962A773A784A795A7B9
:1038900027CFC8010E94620E44E050E0B601C80183
:1038A0000E94430EF70162A173A184A195A10E9419
:1038B000B73962A373A384A395A366A777A780AB48
:1038C00091AB0ECFC8010E94620EB82EBB2009F446
:1038D00007CFC8010E94620EBA94F8CF89A5E3967B
:1038E0000FB6F894DEBF0FBECDBFDF91CF911F9111
:1038F0000F91FF90EF90DF90CF90BF90AF909F908F
:103900008F907F906F905F904F903F902F90089591
:103910007F928F929F92AF92BF92CF92DF92EF925F
:10392000FF920F931F93CF93DF93CDB7DEB7A69788
:103930000FB6F894DEBF0FBECDBF8C01762E942E4D
:10394000852E20E2B22ECE0101967C01FC012B2DAA
:1039500011922A95E9F781E592E09AA389A38FEF66
:103960008BA38CA38DA38EA3680183E4C80ED11C06
:1039700043E450E0BE016F5D7F4FC6010E94B61167
:10398000019609F4BFC081E089838A8386E0A82E6E
:10399000AB821C82F80164817581868197810E94C7
:1039A000B7396D837E838F83988789869A8680E86E
:1039B00090E09C878B874CE150E0B701C6010E94E4
:1039C0002D10F7012B2D11922A95E9F7480188E077
:1039D000880E911CF401D70101900D92AA94E1F791
:1039E00040E150E0B701C6010E942D10F70111928D
:1039F000BA94E9F796E0A92EB12C40E250E0B70165
:103A0000C6010E942D10F1E0AF1AB108B1F783E6AC
:103A1000898392E89A8393E59B838C8385E38D83E6
:103A200081E08E837F829DE3988797E099878A87DC
:103A300086E0F401DE011B9601900D928A95E1F774
:103A40008CE0898B8A8B66ED72E0CE0143960E94F2
:103A5000FE39F8014385BE01675E7F4FC8010E94B1
:103A6000AD1AF8014485BE01655E7F4FC8010E9412
:103A7000AD1AF8014585BE01635E7F4FC8010E9403
:103A8000AD1A4EE150E0B701C6010E942D10F3E0DF
:103A90007F121EC082E3898384E08A83F8019685C1
:103AA0009B8397859C8390899D8391899E8396E3D0
:103AB0009F838887828D8987838D8A87848D8B8772
:103AC000858D8C874CE050E0B701C6010E942D1017
:103AD00087E3898386E08A8391E09B8393E09C83DC
:103AE0008D838FE08E838AE38F838BE388878FEFCC
:103AF000898749E050E0B701C6010E942D10C60138
:103B00000E946D11A6960FB6F894DEBF0FBECDBF12
:103B1000DF91CF911F910F91FF90EF90DF90CF90A9
:103B2000BF90AF909F908F907F9008952F923F927B
:103B30004F925F926F927F928F929F92AF92BF92BD
:103B4000CF92DF92EF92FF920F931F93CF93DF9369
:103B5000CDB7DEB765970FB6F894DEBF0FBECDBF09
:103B60007C016B013A01FB0120E080E090E06AE01B
:103B70003191332309F140ED430F4A3080F4689FBF
:103B8000A001699F500D1124CA01C097830F911D98
:103B900037FD9A958F3F910559F350F313C03E328C
:103BA00089F4233079F0D301A20FB11D12968C93C2
:103BB0002F5F80E090E0DCCF233021F4F301858398
:103BC00081E021C0F7014281538164817581809138
:103BD0005A0690915B06A0915C06B0915D0648176D
:103BE00059076A077B0709F49EC10E94B318870131
:103BF000085F1F4F6F7077277C5FC8010E94ED1030
:103C0000813019F080E090E0F3C181E592E09A8381
:103C10008983F70182819381A481B5818B839C8301
:103C2000AD83BE8345E350E0BE016F5F7F4FC801A7
:103C30000E94B611892B19F4C12CD12C6FC10E949E
:103C4000B318F701778366837627672776277A8309
:103C5000698342E050E0BE016F5F7F4FC8010E9460
:103C60002D1081E090E09E878D8742E050E0BE01FC
:103C7000635F7F4FC8010E942D1080E091E09E8716
:103C80008D8742E050E0BE01635F7F4FC8010E9414
:103C90002D101E861D8642E050E0BE01635F7F4FFF
:103CA000C8010E942D1042E050E0BE01635F7F4FCB
:103CB000C8010E942D1042E050E0BE01635F7F4FBB
:103CC000C8010E942D105601F5018081882311F151
:103CD000F6015F018191811115C045018C189D0885
:103CE0001814190494F48F8641E050E0BE01615F1E
:103CF0007F4FC8010E942D10A401B601C8010E9487
:103D00002D1003C08E3229F7E8CF6501FFEFCF1ADF
:103D1000DF0ADACF1F8641E050E0BE01615F7F4FCE
:103D2000C8010E942D10C12CDD24D394DE86CD86DF
:103D300042E050E0BE01635F7F4FC8010E942D103A
:103D4000DE86CD8642E050E0BE01635F7F4FC80152
:103D50000E942D10C8010E946D11892B09F46CCFAF
:103D600063E0A62EB12CF2E06F0E711C0E94B31816
:103D70001B012C01C8010E948B0E18161906A4F015
:103D80000E94B318DC01CB0182199309A409B5097B
:103D900089389341A105B105D0F462E370E080E079
:103DA00090E00E947918E6CFF70142815381648147
:103DB0007581808D918DA28DB38D481759076A0743
:103DC0007B0741F4848D958DC59721F406C02FEFB4
:103DD0003FEF9AC02EEF3FEF97C0F70181A192A16C
:103DE0000C970CF4A6C04CE050E0BE016F5F7F4F13
:103DF000C8010E94430E8B8190E0982F88272C8168
:103E0000822B9A8B898B298130E0322F22274A819D
:103E1000242BF701468157814217530709F086C0CA
:103E200097FF84C08F709270892B09F0DEC0CF801D
:103E3000D12CDC2CCC248885C82AC114D10409F4E7
:103E4000D1C0812C912C8D8190E0982F88272E81D4
:103E5000822B8816990608F46FC0812C912C41E0C2
:103E600050E0BE016D5E7F4FC8010E94430E8B89FA
:103E7000982F907C09F093C0811186C08B898111A5
:103E8000EECF42E050E0BE01615F7F4FC8010E946B
:103E9000430E42E050E0BE01635F7F4FC8010E94C5
:103EA000430EC8010E94620EC8010E94620EC80142
:103EB0000E94620EC8010E94620E42E050E0BE0104
:103EC0006F5E7F4FC8010E94430E8F8598898115D0
:103ED000914009F069C02D853E853227232732277E
:103EE0002130310509F060C089899A898115944093
:103EF00009F075C044E050E0B301C8012C8B3D8B44
:103F00000E94430E2C893D896901F1E0AF1AB10886
:103F100029F02FEFC216D20609F428CFC8010E945B
:103F2000D810C60165C08EEF9FEF62C02CEF3FEF47
:103F3000EBCF2DEF3FEFE8CF41E050E0BE01635FF4
:103F40007F4FC8010E94430E8D85811113C08D855E
:103F50008111F2CFC8010E94620EC8010E94620E58
:103F6000C8010E94620EC8010E94620EFFEF8F1A04
:103F70009F0A69CF8D859FEF980F9D87882339F31E
:103F8000C8010E94620EF6CF8B899FEF980F9B8B22
:103F9000882309F473CFC8010E94620EF5CFC801CF
:103FA0000E94620E1B8A6ACF412C512C89899A8902
:103FB0009827892798274816590638F4C8010E947F
:103FC000620E8FEF481A580AF1CFEFEF8E1A9E0A51
:103FD0008C149D0409F043CF26EF3FEF95CF27EFD8
:103FE0003FEF92CF2AEF3FEF8FCF2BEF3FEF8CCFFA
:103FF00065960FB6F894DEBF0FBECDBFDF91CF91AF
:104000001F910F91FF90EF90DF90CF90BF90AF90F6
:104010009F908F907F906F905F904F903F902F90E8
:1040200008952F923F924F925F926F927F928F925C
:104030009F92AF92BF92CF92DF92EF92FF920F9337
:104040001F93CF93DF93CDB7DEB727970FB6F894C2
:10405000DEBF0FBECDBF8C010E9487332FEC37E04F
:1040600040E050E00E941A38DC01CB010196A11D0E
:10407000B11DF80184839583A683B78380839183E0
:10408000A283B3835801F3E4AF0EB11CC5010E94B3
:10409000D81064E470E0C5010E94ED10882309F493
:1040A0003CC10E94B3182B013C01812C912C1D8234
:1040B000C8018E5B9F4F9F838E8343E0342E58EE62
:1040C000C52E53E0D52EE12CF12C62E0262EAE81D8
:1040D000BF818C91833009F407C1811120C0F801A0
:1040E00084819581A681B7810196A11DB11D84832C
:1040F0009583A683B7830E94B3186419750986094E
:104100009709A70196010E94F837A90161E0C8014B
:104110000E94881C81E0AE81BF818C93C6C0843030
:10412000F9F4F80184819581A681B7810196A11DDA
:10413000B11D84839583A683B7830E94B318641945
:10414000750986099709A70196010E94F837A90108
:1041500063E0C8010E94881CAE81BF812C92A5C07B
:10416000813061F5F80142AD53AD64AD75AD9E018E
:104170002F5F3F4FC8010E94C21A8D83823009F021
:1041800094C089819A81AB81BC81F8018483958335
:10419000A683B7830E94B318641975098609970925
:1041A000A70196010E94F837A90163E0C8010E94A7
:1041B000881CED81AE81BF81EC937EC0823009F016
:1041C00074C0D801DA964D915D916D917C91DD9727
:1041D0009E012F5F3F4FC8010E94C21A8D83853018
:1041E00009F05CC0EE81FF813082F80182A193A1C9
:1041F000A4A1B5A1892B8A2B8B2B41F484E893E0F1
:10420000A0E0B0E082A393A3A4A3B5A3F80186A184
:1042100097A1A0A5B1A5892B8A2B8B2B61F482A134
:1042200093A1A4A1B5A1B695A7959795879586A3C7
:1042300097A3A0A7B1A7F80182A593A5A4A5B5A5AA
:10424000892B8A2B8B2BA9F482A193A1A4A1B5A1C0
:10425000AC01BD0123E076956795579547952A9562
:10426000D1F7841B950BA60BB70B82A793A7A4A726
:10427000B5A7F80186A197A1A0A5B1A586A797A784
:10428000A0ABB1AB82A593A5A4A5B5A582AB93AB1A
:10429000A4ABB5AB88248394912C0EC0FD81F6307D
:1042A00021F4AE81BF811C9207C0BD81BF3F21F4C4
:1042B000EE81FF8110821D82F1E08F16910409F4D6
:1042C00006CF0E94B318DC01CB0184199509A60919
:1042D000B709F80126A937A940AD51AD281739070C
:1042E0004A075B0708F0F3CEC5010E94D810F80119
:1042F00084819581A681B7810196A11DB11D84831A
:104300009583A683B7830E94B318F801FE96608355
:10431000718382839383C40102C080E090E027967A
:104320000FB6F894DEBF0FBECDBFDF91CF911F91C6
:104330000F91FF90EF90DF90CF90BF90AF909F9044
:104340008F907F906F905F904F903F902F90089547
:1043500063E080E00E9445276AE876E08EE596E01B
:104360000C943A1563E080E00E94452769E776E007
:104370008EE596E00C943A150F931F93CF93DF933D
:104380000EE011E0C0E0D0E0F80161918F01CE01B4
:104390000E94DA372196C633D105B1F780E090E06C
:1043A0000E94D23790910E0189130AC062ED76E027
:1043B00087EA95E0DF91CF911F910F910C9402163F
:1043C000DF91CF911F910F910895CF93C82F682F40
:1043D000607F8EE596E00E94C20C80E1C89FB0012C
:1043E00011248EE596E0CF910C94C20C81E00E94DE
:1043F000E5218BE39FE10197F1F70895CF93C82F53
:10440000462F61E070E00E943D1161E070E08C2F6A
:104410000E9447118111F9CFCF910895CF93DF9377
:10442000EC0181E592E0998388831A821B821C82C9
:104430001D8280E590E00E943E26BE016E5F7F4FA8
:1044400044E050E08FE090E00E94150D0E943D2670
:10445000CE01DF91CF9108958F929F92AF92BF923C
:10446000CF92DF92EF92FF920F931F93CF93DF9340
:10447000B82E4B018A01A22E68E270E00E9447111B
:10448000C82FD0E069E270E08B2D0E944711DC2F2D
:10449000CC27C82B9E013770CB2CD12CC601880F9E
:1044A000991FAC0141565A4F6A01FA0180819181EE
:1044B000820F931FA801420F531F4130584098F0BC
:1044C00060E078E07B01E21AF30AA701B4010E94E0
:1044D000150DA8014E195F09B4016E0D7F1DF6017F
:1044E0008081918102C0A801B4010E94150DA11024
:1044F0000EC0C00FD11F4D2F68E270E08B2D0E94BF
:104500003D114C2F69E270E08B2D0E943D11DF912F
:10451000CF911F910F91FF90EF90DF90CF90BF90C0
:10452000AF909F908F9008959F92AF92BF92CF923D
:10453000DF92EF92FF920F931F93CF93DF93982E0A
:104540008B015A01690164E270E00E944711E82E74
:10455000F12C65E270E0892D0E944711FE2CEE24BB
:10456000E82AE701C00FD11F9E013770E92CF12C1A
:10457000C701880F991FAC0149565A4F7A01FA01B9
:1045800080819181820F931FA9014C0D5D1D4130E7
:10459000584090F000E018E0021B130BA801B50191
:1045A0000E94450DA601401B510BB501600F711F04
:1045B000F7018081918102C0A601B5010E94450DDD
:1045C000CC0DDD1D4D2F64E270E0892D0E943D1160
:1045D0004C2F65E270E0892DDF91CF911F910F91F3
:1045E000FF90EF90DF90CF90BF90AF909F900C9492
:1045F0003D11FF920F931F93CF93DF93F82EC0E0EE
:10460000D0E08F2D0E94F60C8C01892B21F08F2D8C
:104610000E94F60CEC01C017D10799F7CE01DF918B
:10462000CF911F910F91FF9008953F924F925F920B
:104630006F927F928F929F92AF92BF92CF92DF92B2
:10464000EF92FF920F931F93CF93DF9300D000D090
:10465000CDB7DEB720910D01233021F02F3F09F0B7
:104660002CC204C0E1EDF6E0349076C023E0209344
:104670000D01E1EDF6E0E491EF3F09F41EC2E130F7
:1046800011F1E23009F443C0E11165C014BC15BC5E
:1046900024B5226024BD25B5216025BDE0ECF6E0FF
:1046A000E491F0E0EE0FFF1FED54F94F25913491A6
:1046B00030938F0620938E06E2EAF6E0E491E093D1
:1046C0008D06312C4BC010928000109281002091F9
:1046D0008100286020938100209181002160209337
:1046E0008100E0ECF6E0E491F0E0EE0FFF1FED5406
:1046F000F94F2591349130938C0620938B06E2EA92
:10470000F6E0E491E0938A063324339427C01092B4
:10471000B0001092B1002091B00022602093B00050
:104720002091B10021602093B100E0ECF6E0E4912B
:10473000F0E0EE0FFF1FED54F94F259134913093C7
:10474000920520939105E2EAF6E0E491E09390056A
:10475000B2E03B2E03C03E2E37FCAFC12A013B0125
:104760008C0161E083E00E943D184801A12CB12C2E
:10477000832D8D7F09F0BBC060E072E18AE790E095
:10478000A50194010E941A3829833A834B835C83E4
:1047900069017A0121E0C21AD108E108F1088FEF1E
:1047A000C816D104E104F10409F008F44CC060E437
:1047B00072E48FE090E0A50194010E941A3869012B
:1047C0007A01E1E0CE1AD108E108F108F2E03F12E7
:1047D00020C02FEFC216D104E104F10409F008F45F
:1047E0006AC160E970ED83E090E0A50194010E9448
:1047F0001A3869017A0181E0C81AD108E108F10884
:10480000EFEFCE16D104E104F10409F0D0F583E016
:1048100067C0FFEFCF16D104E104F104B1F0A8F0B6
:1048200068E478EE81E090E0A50194010E941A38D6
:1048300069017A0181E0C81AD108E108F108332042
:1048400009F4DFC02FC181E001C082E03320A1F074
:1048500047C089819A81AB81BC812AE0B595A79533
:10486000979587952A95D1F76C017D0121E0C21AB1
:10487000D108E108F10885E095B5987F892B85BDC1
:104880006FC068E478EE81E090E0A50194010E9499
:104890001A3869017A01F1E0CF1AD108E108F1086C
:1048A0002FEFC216D104E104F10409F008F4A7C007
:1048B00064E274EF80E090E0A50194010E941A3850
:1048C00069017A01E1E0CE1AD108E108F108FFEFB1
:1048D000CF16D104E104F10411F008F0B4C085E072
:1048E0009091B100987F892B8093B10039C060E02E
:1048F00072E18AE790E0A50194010E941A386901EB
:104900007A0181E0C81AD108E108F108C114D10484
:10491000E1E0EE06F10488F068E478EE81E090E0F2
:10492000A50194010E941A3869017A01F1E0CF1AB9
:10493000D108E108F10893E001C091E021E03212D2
:104940000FC080918100887F892B80938100411462
:1049500051046104710449F42FEF3FEFA9012DC008
:10496000411451046104710471F0D801AA0FBB1FF6
:10497000A30192010E94393828EE33E040E050E074
:104980000E94F83703C02FEF3FEFA90181E03816EE
:10499000A1F0E2E03E1619F131108FC0C7BC2093A0
:1049A000940630939506409396065093970680910F
:1049B0006E00826080936E0080C0D0928900C092A9
:1049C000880020939006309391064093920650936E
:1049D000930680916F00826080936F006EC0C092DA
:1049E000B30020939305309394054093950550931D
:1049F0009605809170008260809370005EC084E0B4
:104A00006FCFFFEFCF16D104E104F104D1F0C8F06D
:104A100062E17AE780E090E0A50194010E941A38F3
:104A200069017A0181E0C81AD108E108F108EFEFC5
:104A3000CE16D104E104F10411F008F00ACF84E0AD
:104A40001BCF83E019CF62E17AE780E090E0A50117
:104A500094010E941A3869017A0181E0C81AD108CC
:104A6000E108F108EFEFCE16D104E104F104C1F042
:104A7000B8F089819A81AB81BC814AE0B595A79550
:104A8000979587954A95D1F76C017D0121E0C21A6F
:104A9000D108E108F108332009F4EDCE87E020CFFA
:104AA00086E0D4CEFFEFCF16D104E104F10409F083
:104AB00050F684E0CBCE82E013CF0F900F900F9092
:104AC0000F90DF91CF911F910F91FF90EF90DF90AA
:104AD000CF90BF90AF909F908F907F906F905F909E
:104AE0004F903F900895CF93DF931F92CDB7DEB7DD
:104AF0006983DC01ED91FC910280F381E02D41E0BE
:104B000050E0BE016F5F7F4F09950F90DF91CF910D
:104B10000895DC01ED91FC91068CF78DE02D09954F
:104B200091E089270895862F089581E086270895CA
:104B3000089580E090E00895FC0184850C94F00DC8
:104B4000CF93DF931F92CDB7DEB741E050E0BE01B7
:104B50006F5F7F4FFC0184850E94F00D18161906C7
:104B60001CF4898190E002C08FEF9FEF0F90DF91DE
:104B7000CF910895FC018485843011F00C94CE0D02
:104B800080E090E00895CF92DF92EF92FF920F9332
:104B90001F93CF93DF93CDB7DEB7AF970FB6F894DF
:104BA000DEBF0FBECDBF7C016A0101E512E01A83B2
:104BB00009831C861B8688EE93E0A0E0B0E08D8719
:104BC0009E87AF87B88B89E891E09A878987188F8D
:104BD0000F8B198E1A8E1B8E1C8E84E089A31DA349
:104BE0000CA31EA21FA218A619A68091520690918E
:104BF0005306A0915406B09155068CA79DA7AEA769
:104C0000BFA78B839C83AD83BE8318861F82AE01B2
:104C10004C5D5F4FCE0101960E94961D813091053B
:104C2000B1F4D701ED91FC910684F785E02D1BA727
:104C30000AA78EA19FA1A8A5B9A58CA79DA7AEA7DD
:104C4000BFA7A601BE01665D7F4FC7010995AF965C
:104C50000FB6F894DEBF0FBECDBFDF91CF911F918D
:104C60000F91FF90EF90DF90CF90089544E050E0D7
:104C7000BC018FE090E00C94450D08958CBD9DBD66
:104C800008958F929F92AF92BF92CF92DF92EF9250
:104C9000FF920F931F93CF936C015B017A01FC018C
:104CA000C485C43041F481E090E0F60193838283AF
:104CB00080E090E04EC08A014130584010F000E0A2
:104CC00018E080E590E00E943E268C2F0E94F92299
:104CD0004C0163E070E08C2F0E944711873111F086
:104CE0008C3121F48016910660F302C000E010E0E0
:104CF00080E590E00E943E269801A50160E070E00A
:104D00008C2F0E94942260E270E08C2F0E94FE2182
:104D100062E070E08C2F0E94471184FD10C063E0B8
:104D200070E08C2F0E944711811104C08C2F0E94CB
:104D3000E40EB9CF80E590E00E943E26E9CF40E145
:104D400062E070E08C2F0E943D11012B09F4ABCF83
:104D5000C701CF911F910F91FF90EF90DF90CF90FF
:104D6000BF90AF909F908F900895CF92DF92FF9267
:104D70000F931F93CF93DF93FC012485243009F018
:104D800077C06A01EB018C01F12C8F2D0E94B30FCB
:104D9000811103C0F801F48607C08B7F8831D1F3FD
:104DA000F394F4E0FF12F1CFF8018485843009F424
:104DB0005FC020914401309145012F5F3F4F11F4B6
:104DC00020E030EC309345012093440140914401B0
:104DD0005091450120E061E00E94F80EF801F48452
:104DE0008A818F3F51F48B818F3F91F48C818F3F6B
:104DF00079F48D818F3F61F438C0811109C08B81B6
:104E0000811106C08C81811103C08D81882369F1D5
:104E1000C114D10451F180E590E00E943E26BE010C
:104E20006E5F7F4F8F2D90E0982F882744E050E0F1
:104E3000845F9B4F0E94450DB6018F2D0E94A511E6
:104E400064E070E08F2D0E94FE21C8010E94F611DF
:104E5000873189F061E070E080E090E00E9479188D
:104E6000C8010E94F6118111F0CF84E0F801848717
:104E700080E090E002C081E090E0DF91CF911F914F
:104E80000F91FF90DF90CF900895CF93DF93CDB730
:104E9000DEB728970FB6F894DEBF0FBECDBF98E0FF
:104EA000E9E5F2E0DE01119601900D929A95E1F7A5
:104EB00090916706961710F46FEF690FFE01319617
:104EC000E60FF11DE60FF11D9081890F806828968D
:104ED0000FB6F894DEBF0FBECDBFDF91CF910C941B
:104EE000E521CF92DF92EF92FF920F931F93CF9322
:104EF000DF936B01770FEE08FF08F7FE1BC0EC0194
:104F00006DE20E9433158C0144275527BA014C19D4
:104F10005D096E097F092AE0CE010E947315800F9A
:104F2000911FDF91CF911F910F91FF90EF90DF9034
:104F3000CF9008952AE0B701A601DF91CF911F918C
:104F40000F91FF90EF90DF90CF900C9473158091AC
:104F5000460120E4829FC001112480937C0080914F
:104F60007A00806480937A0080917A0086FDFCCF7D
:104F7000809178002091790090E0922B0895CF9352
:104F8000DF93CDB7DEB761970FB6F894DEBF0FBEE3
:104F9000CDBF789484B5826084BD84B5816084BDC2
:104FA00085B5826085BD85B5816085BD80916E00C7
:104FB000816080936E0010928100809181008260F8
:104FC0008093810080918100816080938100809135
:104FD00080008160809380008091B1008460809324
:104FE000B1008091B00081608093B00080917A0020
:104FF000846080937A0080917A00826080937A0046
:1050000080917A00816080937A0080917A00806834
:1050100080937A001092C100E091B705F091B80535
:1050200082E08083E091B305F091B4051082E091B5
:10503000B505F091B60580E180831092BF05E0913F
:10504000BB05F091BC0586E08083E091B905F09145
:10505000BA05808180618083E091B905F091BA053D
:10506000808188608083E091B905F091BA058081E4
:1050700080688083E091B905F091BA0580818F7DC9
:10508000808369E271E087EA95E00E943A1561E663
:1050900072E087EA95E00E94F81667EF70E087EA11
:1050A00095E00E94021683E08093460160E082E072
:1050B0000E943D1860E08EE00E943D1861E084E0AF
:1050C0000E943D1861E083E00E943D1862E085E0A7
:1050D0000E943D1880E090E00E94D23790910E012E
:1050E000891799F10E948C071092E4021092E30252
:1050F0001092E2021092E1021092E00281E08093AD
:10510000DF021092DE0261E082E10E948B1761E013
:1051100083E10E948B178091B9008E7F8093B90044
:105120008091B9008D7F8093B90088E48093B800A6
:1051300085E48093BC0010926306809167068230FC
:10514000B0F098E09093630612C0AEE0EA2EA1E0C2
:10515000FA2E00E010E0C8010E94D237D7018D93EB
:105160007D010F5F1F4F06331105A9F7BBCF90914B
:105170006806992339F0813029F4809163068460B0
:105180008093630662E370E080E090E00E9479180B
:10519000609169068EE596E00E945D0C68EE73E012
:1051A00080E090E00E94791860E38EE596E00E942E
:1051B000C20C0BE416E4C8010197F1F760E38EE539
:1051C00096E00E94C20CC8010197F1F760E38EE5FA
:1051D00096E00E94C20C83E592E00197F1F760E24D
:1051E0008EE596E00E94C20C8091630680620E9468
:1051F000E52184E0809364068CE00E94E5210E9412
:10520000F62182E08093650686E00E94E52182E037
:105210000E94E5218BE39FE10197F1F788E08093FD
:10522000690660E08EE596E00E945D0C81E0809367
:10523000060160E085E00E9445276FED70E08EE595
:1052400096E00E943A1561E672E08EE596E00E94D3
:10525000F81661E080E00E9445276AEC70E08EE578
:1052600096E00E943A1562E089E00E94452766ECCC
:1052700070E08EE596E00E943A1563E080E00E94BF
:10528000452761EB70E08EE596E00E943A150091AB
:105290000001109101011016110634F485E00E94FE
:1052A0006217892B09F049C00E94F621F8941092E8
:1052B000800010928100109285001092840088E096
:1052C0009DE390938900809388008091810088609D
:1052D000809381008091810085608093810080911E
:1052E0006F00826080936F008CE993E090930301DC
:1052F0008093020180916900836080936900E89A3D
:10530000789445E150E060E270E081EF92E00E9425
:10531000D8391092050385E00E94621721E0892B9D
:1053200009F420E020930B01211114C066EE70E017
:1053300087EA95E00E9402160DC0045611091093E9
:1053400001010093000164E670E080E090E00E94BB
:1053500079189DCF80913A01882321F061E084E0A3
:105360000E948B1722242A94322CE8EE8E2EE3E042
:105370009E2EA12CB12CF1E1CF2EF2E0DF2E87EA98
:1053800095E00E941F147C01892B69F187EA95E062
:105390000E94FD138A3089F08D30B9F020916503A9
:1053A00030916603F901E75DFC4F80832F5F3F4F2B
:1053B000309366032093650308C089E293E00E945E
:1053C000230A1092660310926503E0916503F09141
:1053D0006603E75DFC4F10826AE070E080E090E0D9
:1053E0000E947918CCCF85E00E946217019709F4DA
:1053F00064C164EF71E080E090E00E94791885E07C
:105400000E946217892B19F082E090E002C081E0CF
:1054100090E09093E6028093E5028091060181116D
:1054200002C00E94250480913E0190E090930A0101
:1054300080930901809107019091080197FF07C0AF
:105440008091E5029091E602019709F48BC4809166
:10545000E5029091E6020297F9F40E94F62180910C
:1054600007019091080197FF0AC001978B3FBFEF9A
:105470009B074CF430920801209207010DC0019661
:10548000873091052CF4909308018093070104C0A4
:105490001092080110920701009107011091080174
:1054A00017FDFBC00E94F6210730110508F0F5C07A
:1054B000F801EC5CFF4F0C94B1392091E50230917A
:1054C000E60281E090E02130310511F080E090E0CB
:1054D000919581959109909308018093070164EE5D
:1054E00071E08EE596E00E943A1563E080E00E944C
:1054F000452765ED71E08EE596E00E943A158091B2
:10550000070190910801019609F0C7C00E94F62199
:10551000C4C065EC71E08EE596E00E943A1563E048
:1055200080E00E9445278091E5029091E602019774
:1055300049F40E948C0710928500109284006CEB55
:1055400071E08DC06CEA71E08AC08091E5029091B3
:10555000E602019731F490913D0181E08927809323
:105560003D0165EA71E08EE596E00E943A1561E042
:1055700080E00E94452780913D0155C08091E50261
:105580009091E602019751F480913E01865F893740
:1055900018F480933E0102C010923E016FE871E062
:1055A0008EE596E00E943A1561E080E00E94452772
:1055B00040913E01442349F050E060E070E02AE071
:1055C0008EE596E00E94731506C06EE971E08EE5E7
:1055D00096E00E943A150E94B2215FC08091E502D8
:1055E0009091E602019799F490913A0181E0892720
:1055F00080933A01882349F00E947D0821E0892B9D
:1056000009F420E02093270302C0109227036BE7E0
:1056100071E08EE596E00E943A1561E080E00E941C
:10562000452780913A01882381F262EA71E0CFCF69
:105630006BE671E08EE596E00E943A1563E080E04B
:105640000E9445278091E5029091E602019729F496
:105650000E94BC2164E671E002C065E571E08EE560
:1056600096E00E943A1519C063E471E08EE596E079
:105670000E943A1563E080E00E94452760E371E0F4
:105680008EE596E00E943A158091E5029091E6023F
:10569000019719F481E00E94FB0385E00E946217E4
:1056A000892B39F462E370E080E090E00E94791881
:1056B000F4CF1092E6021092E50280910C0188234B
:1056C00009F4B1C08CE892E00E94F206BC0187EABE
:1056D00095E00E945E1565E672E087EA95E00E941B
:1056E0005E158091090190910A01181619063CF087
:1056F00080913E01882319F080E00E94FB03109204
:105700000C01009107011091080117FF8CC00E9445
:10571000A727BC01990F880B990B0E94B53620E092
:1057200030E048EC52E40E9414372B013C016091B8
:105730003F0170E080E090E00E94B5369B01AC0133
:10574000C301B2010E94FF3820E030E044EB53E493
:105750000E94AE3687FD11C30E94A727BC01990F96
:10576000880B990B0E94B53620E030E048EC52E4FB
:105770000E9414372B013C0160913F0170E080E0F2
:1057800090E00E94B5369B01AC01C301B2010E94BA
:10579000FF3820E030E04CED53E40E94A7391816A2
:1057A0000CF4EBC210921A0360E080E00E944527DF
:1057B0000E5F1F4F02301105B8F40E944F04E6E05F
:1057C000F3E001900020E9F73197BF016650734084
:1057D0006F507D4F8EE596E00E94F81666E073E00C
:1057E0008EE596E00E94F8168091070190910801DD
:1057F0008D3FFFEF9F0709F461C50CF003C38B3F9A
:105800003FEF930709F42BC6049609F4BCC5209119
:105810001B0330911C0380913B0190913C01821746
:10582000930708F449C680912803882339F18091B1
:105830003D01882399F020911B0330911C03809136
:105840003B0190913C012817390740F44AE050E0B1
:1058500060E070E080E991E00E94152361E084E05F
:105860000E948B1764E670E080E090E00E94791857
:1058700060E084E00E948B171092280380910B0156
:10588000882309F40AC180912703882309F4FDC005
:1058900080913A01882309F400C184E896E00E94CF
:1058A000D7120DE113E0712C1C821B828D829E8227
:1058B000AF82B886DA82C9827D86F8012191319162
:1058C0008F01809188069091890628173907F1F495
:1058D000CE0101960E94F611873111F08C31B1F49E
:1058E000CE0101960E94BA25892B81F0EB80FC80C5
:1058F0008D819E81AF81B88529853A854B855C85F0
:105900002E873F87488B598B7D8408C0739434E081
:105910007312CACF88EE93E0A0E0B0E0F0927A066E
:10592000E092790680937B0690937C06A0937D0697
:10593000B0937E068E859F85A889B98980937F065E
:1059400090938006A0938106B0938206709283069E
:1059500094E0791609F4A1C01092940311E087E74E
:1059600096E00E946B12882309F48AC087E796E0CC
:105970000E94BA25892B09F47CC087E796E00E9433
:10598000A0258D3009F064C06CE673E087EA95E0ED
:105990000E94F8168CE693E09A838983AE014F5FEC
:1059A0005F4F6DE772E00E94D234AE014F5F5F4FF0
:1059B0006CE872E089819A810E94D234DC012C91DA
:1059C000222329F00E94230A811110936B03ECE635
:1059D000F3E001900020E9F7EE56F340A1F562E410
:1059E00073E087E796E00E943A15809125038823AB
:1059F00019F061E273E002C066E073E087E796E0C9
:105A00000E943A1560EF72E087E796E00E943A152F
:105A100080912503882329F087E796E00E940605F8
:105A20000DC080916B03882319F06DEE72E002C007
:105A300064EE72E087E796E00E940216109225035A
:105A400010926B031DC01092940310926C0311C04E
:105A5000E0919403AE2FB0E0A459BC4F8C93EF5F5C
:105A6000E83208F0E7E2E0939403F0E0E459FC4FF9
:105A7000108261E070E080E090E00E9479186FCFC2
:105A800087E796E00E948F1208C00E947D0821E0FF
:105A9000892B09F420E02093270380912603882393
:105AA00009F45DC180912703882309F456C16EE78C
:105AB00073E087EA95E00E943A1565E171E0CE0156
:105AC00001960E94FA1640E550E0BE016F5F7F4FDD
:105AD0008AE696E00E94B526892B09F442C069E760
:105AE00073E08AE696E00E943A1569E171E08AE681
:105AF00096E00E94F81667E773E08AE696E00E9457
:105B00003A158FE792E00E94F206BC018AE696E021
:105B10000E94F8166BE673E08AE696E00E94021691
:105B200060E673E087EA95E00E9402168AE696E056
:105B30000E94BA25892B81F08AE696E00E94A02572
:105B4000682F87EA95E00E94331561E070E080E0FD
:105B500090E00E947918EACF8AE696E00E948F12C0
:105B600006C064E573E087EA95E00E9402160091A2
:105B70005606109157060115110509F4EEC00E9452
:105B8000B3182B013C017801EEE3EE0EF11CF70196
:105B900080819181A281B381A3019201281B390BDD
:105BA0004A0B5B0BCA01B901683E33E073078105FC
:105BB000910508F446C028EE33E040E050E00E9432
:105BC000F837461A570A680A790AD7014D925D924A
:105BD0006D927C921397F80186A597A5A0A9B1A90B
:105BE00029013A01440C551C661C771C8415950547
:105BF000A605B70528F416A617A610AA11AA09C06B
:105C0000821B930BA40BB50BF80186A797A7A0AB3B
:105C1000B1ABF80182A993A9A4A9B5A984159505EA
:105C2000A605B70528F412AA13AA14AA15AA09C032
:105C3000821B930BA40BB50BF80182AB93ABA4AB07
:105C4000B5ABF80186A597A5A0A9B1A9892B8A2B88
:105C50008B2B61F4EE5BFF4F8081833039F484E05D
:105C60008083C8010E941120019602C080E090E06C
:105C7000D801D2964D915D916D917C91D597452B30
:105C8000462B472BA1F4F801EE5BFF4F2081233018
:105C900011F021110CC01082F8013E9684E1DF0161
:105CA0001D928A95E9F7C8010E941120039682305F
:105CB000910519F0049709F050C080E590E00E942A
:105CC0003E266091560670915706625F7F4FCE0167
:105CD00001960E94FA16CE0103960E943626609124
:105CE0005606709157066A5E7F4FCE0101960E945C
:105CF000FA1644E050E0BE016D5F7F4F81E090E016
:105D00000E94450D60915606709157066E5E7F4F5A
:105D1000CE0101960E94FA1644E050E0BE016D5F8C
:105D20007F4F85E090E00E94450D0E943D266091E6
:105D3000560670915706625E7F4FCE0101960E9413
:105D4000FA168B819C81AD81BE818093520690931F
:105D50005306A0935406B0935506109226030E9452
:105D6000BF140DCB10920801109207011092E602A9
:105D70001092E5020E94F6216ACB0E94F62161E0B2
:105D800080E00E9445276AED72E08EE596E00E9471
:105D90003A1562E080E00E9445276BEC72E08EE5E8
:105DA00096E00E943A150E94A727BC01990F880B24
:105DB000990B0E94B53620E030E048EC52E40E9496
:105DC00014372B013C0160913F0170E080E090E0CE
:105DD0000E94B5369B01AC01C301B2010E94FF389D
:105DE000AB01BC0120E030E08EE596E00E94161683
:105DF00068EC72E08EE596E00E943A1581E08093AF
:105E00001A0311CD8E3F5FEF950709F4A5C10196E6
:105E100009F0FDCC60E080E00E94452780912703D7
:105E20008823D9F065E171E0CE0101960E94FA164F
:105E300040E550E0BE016F5F7F4F8AE696E00E942A
:105E4000B526892B51F08AE696E00E948F126BED01
:105E50008EE596E00E94DB0C06C06091F1028EE5B3
:105E600096E00E94331561E080E00E94452764EED1
:105E70008EE596E00E94DB0C64EC72E08EE596E025
:105E80000E943A1561E084E00E94452760911B035F
:105E900070911C0380E090E00E94B3362091400195
:105EA0003091410140914201509143010E94FF38DD
:105EB00060936703709368038093690390936A0308
:105EC00020E030E040E251E40E94AE3687FF06C099
:105ED0006091F1028EE596E00E94331540916703D0
:105EE000509168036091690370916A0322E030E089
:105EF0008EE596E00E94161661E08BE00E94452731
:105F00006FEB72E08EE596E00E943A1561E08FE05B
:105F10000E9445276091EF027091F00280E090E0CE
:105F20000E94B336209140013091410140914201DD
:105F3000509143010E94FF38609367037093680398
:105F40008093690390936A0320E030E040E251E4DB
:105F50000E94AE3687FF06C06091F1028EE596E0A2
:105F60000E94331540916703509168036091690363
:105F700070916A0322E030E08EE596E00E941616EA
:105F800062E080E00E9445276AEB72E08EE596E0D1
:105F90000E943A156EEF72E08EE596E00E94F816C8
:105FA00062E084E00E94452760911B0370911C030E
:105FB00080E090E00E94B3362B013C0120E030E00D
:105FC00040E251E4609140017091410180914201B1
:105FD000909143010E9414379B01AC01C301B201AF
:105FE0000E94AE3687FF06C06091F1028EE596E012
:105FF0000E94331540911B0350911C0360E070E038
:106000002AE08EE596E00E94731562E08BE00E9424
:10601000452765EB72E08EE596E00E943A1562E056
:106020008FE00E944527209140013091410140912D
:106030004201509143016091EB027091EC0280911A
:10604000ED029091EE020E94FF3860936703709317
:1060500068038093690390936A0320E030E040E294
:1060600051E40E94AE3687FF06C06091F1028EE5D2
:1060700096E00E9433154091670350916803609148
:10608000690370916A0322E030E08EE596E00E9499
:10609000161663E080E00E94452761EF72E08EE50E
:1060A00096E00E94F81663E080E00E944527809108
:1060B0001B0390911C038E31910518F46EEA72E077
:1060C00022C08B34910518F469EA72E01CC086394D
:1060D000910518F461EA72E016C08039B1E09B07BF
:1060E00018F466E972E00FC0883EE3E09E0718F4FA
:1060F0006DE872E008C0803D974018F463E872E0F4
:1061000002C06BE772E08EE596E00E943A1563E00C
:106110008EE00E94452764E772E08EE596E00E94DB
:106120003A1563E08EE00E9445270BE411E0D801A8
:106130008D919D918D0120911B0330911C0382173D
:10614000930728F46FEF8EE596E00E94DB0CB1E038
:1061500007351B0761F75BCB61E080E00E944527B4
:1061600061EF72E08EE596E00E94F81661E080E053
:106170000E94452769E672E08EE596E00E943A1596
:106180004091E7025091E8026091E9027091EA02C1
:106190002AE08EE596E00E94731562E080E00E949E
:1061A000452761EF72E08EE596E00E94F816609157
:1061B000E7027091E8028091E9029091EA020E9460
:1061C000B3362091400130914101409142015091FC
:1061D00043010E94FF3860936703709368038093C4
:1061E000690390936A0362E080E00E94452763E6BA
:1061F00072E08EE596E00E943A1564EE8EE596E038
:106200000E94DB0C6EE572E08EE596E00E943A1586
:1062100040916703509168036091690370916A032C
:1062200022E030E08EE596E00E94161663E080E002
:106230000E94452761EF72E08EE596E00E94F81615
:106240002091E7023091E8024091E9025091EA0280
:10625000A4E6B0E00E9439380E94B3362091400194
:106260003091410140914201509143010E94FF3819
:1062700060936703709368038093690390936A0344
:1062800063E085E00E94452764EE8EE596E00E947B
:10629000DB0C6AE572E08EE596E00E943A154091CB
:1062A0006703509168036091690370916A0321E06C
:1062B00030E08EE596E00E941616A9CA6CE472E002
:1062C0008EE596E00E943A154091400150914101BF
:1062D000609142017091430122E030E08EE596E04A
:1062E0000E94161661E080E00E9445276EE372E08E
:1062F0008EE596E00E943A150E94A727BC01990FEF
:10630000880B990B0E94B53620E030E048EC52E44F
:106310000E9414372B013C0160913F0170E080E046
:1063200090E00E94B5369B01AC01C301B2010E940E
:10633000FF38AB01BC0120E030E08EE596E00E9422
:1063400016166AE372E08EE596E00E943A1562E066
:1063500080E00E9445276CE272E08EE596E00E94A4
:106360003A1540913B0150913C0160E070E02AE019
:106370008EE596E00E94731566E272E08EE596E087
:106380000E943A1569C06AE172E08EE596E00E94CB
:106390003A1561E080E00E94452765E172E08EE5F4
:1063A00096E00E943A1580913A01882359F0CE0177
:1063B00001960E940E226EE576E0CE0101960E94C3
:1063C000BC1506C061E172E08EE596E00E943A15C8
:1063D00062E080E00E9445276CE072E08EE596E086
:1063E0000E943A154091150150E060E070E02AE00B
:1063F0008EE596E00E9473156AE072E08EE596E005
:106400000E943A154091160150E060E070E02AE0E9
:106410008EE596E00E94731568E072E08EE596E0E6
:106420000E943A154091170150E060E070E02AE0C8
:106430008EE596E00E94731566E072E08EE596E0C8
:106440000E943A154091180150E060E070E02AE0A7
:106450008EE596E00E9473150E94A821D8C96FEFBF
:1064600071E08EE596E00E943A1561E672E08EE5F5
:1064700096E00E94F81661E080E00E94452768E6F9
:1064800072E08EE596E00E94F8166091F1028EE5CA
:1064900096E00E94331564E772E08EE596E00E9474
:1064A000F81663E080E00E9445276AEE71E08EE511
:1064B00096E00E943A15ABC944EF51E060E070E00D
:1064C00088EE93E00E94152380916406982F9460D3
:1064D000909364068C600E94E5219091060181E012
:1064E000892780930601882321F088E0809369063C
:1064F00002C01092690660E08EE596E00E945D0C95
:1065000092C9E8E9F6E081E592E091838083128206
:10651000138214821582E7EAF5E01382128248EEB4
:1065200053E060E070E0448355836683778321EB1A
:1065300031E03183208325EC30E03587248724EC5B
:1065400030E03787268720EC30E0318B208B21EC40
:1065500030E0338B228B22EC30E0358B248B26EC21
:1065600030E0378B268B118E128E138E148EE4E45E
:10657000F6E013821282448355836683778323EC8B
:1065800031E031832083EEE9F6E09183808312824B
:10659000138214821582E4EAF6E0918380831282EA
:1065A000138214821582EAEAF6E0918380831282D4
:1065B000138214821582E0EBF6E0918380831282CD
:1065C000138214821582E0E5F6E0918380831282C3
:1065D000138214821582E8E5F6E0918380831282AB
:1065E000138214821582E6EBF6E091838083128297
:1065F000138214821582ECEBF6E091838083128281
:10660000138214821582E4E8F6E01382128287E393
:1066100092E09183808380E590E095838483E7E72F
:10662000F6E013821282448355836683778321E1E7
:1066300032E03183208384E08487EAE6F6E0138247
:1066400012824483558366837783318320838487D2
:10665000EEE5F6E01382128225ED31E031832083EE
:1066600097E2948394E190878187128688E08387FC
:1066700008958F929F92AF92BF92CF92DF92EF9246
:10668000FF92CF93DF93EC01688179818A819B81AE
:10669000611571058105910521F464E279ED8BE5C1
:1066A00097E02DE133EF41E050E00E941A384901B4
:1066B0005A019B01AC01A7EAB1E40E9439386B0191
:1066C0007C01ACEEB4EFA50194010E944738DC01D7
:1066D000CB018C0D9D1DAE1DBF1DB7FF03C00197E3
:1066E000A109B04888839983AA83BB83BC01CD01EB
:1066F0009F77DF91CF91FF90EF90DF90CF90BF9089
:10670000AF909F908F9008950E943933089587E449
:1067100091E00E94393308956093470170934801D6
:106720008093490190934A010895A6E0B0E0EBE917
:10673000F3E30C944C385C016B017A01611571052F
:1067400019F0DB018D939C93E114F10429F0C7014A
:106750000297839708F0DCC03501BFEF6B1A7B0A04
:10676000F5011081812F90E00E94C934892B11F02E
:106770005301F2CF1D3249F43501F2E06F0E711C66
:10678000D50111961C9101E009C01B3231F435018D
:10679000B2E06B0E711CF501118100E0E114F1040F
:1067A00009F4C4C0F0E1EF16F10489F4103399F54F
:1067B000D3018C918F7D883509F0B2C011961C9160
:1067C000B2E06B0E711C026050E1E52EF12CEAE0A4
:1067D000EE16F10409F4B0C0F0E1EF16F104D9F0BF
:1067E00028E0E216F10451F438E0E32EF12C88247D
:1067F0008A94982CA82C4FE1B42E13C06FEF7FEF32
:10680000CB0197010F2C000C440B550B0E94F8375D
:1068100049015A0106C088248A94982CA82C2FE09C
:10682000B22E7E826D8260E020E030E0A901270177
:106830000F2C000C660877082D803E80E0EDE10FFC
:10684000EA3060F08FEB810F8A3110F4E9EC05C07B
:106850008FE9810F8A3190F5E9EAE10F8E2F90E000
:106860008E159F055CF56F3F09F182169306A4060D
:10687000B506D8F0C301B2010E94E8372E2F30E0F0
:1068800040E050E029833A834B835C83260F371F17
:10689000481F591F89819A81AB81BC81281739070C
:1068A0004A075B0710F061E001C06FEFED81FE81E8
:1068B0003196FE83ED83D1011C91BECFC114D1046A
:1068C00089F0662339F08D819E810197F6019183CD
:1068D000808308C001FF06C08D819E810297D6018A
:1068E0008D939C9300FF07C050954095309521955E
:1068F0003F4F4F4F5F4F67FF10C082E290E0909391
:10690000C7068093C6066FEF7FEF8FEF9FEF1BC028
:1069100060E070E080E090E016C0B901CA0113C0E9
:1069200010E3E114F10409F45FCF51CF103309F4FF
:106930003FCF9AE0E92EF12C89E9882E982CA82CDB
:1069400089E1B82E6ECF2696E2E10C94683866276E
:1069500077270C942635FC0188279927E894219104
:106960002032E9F3293010F02E30C8F32B3241F0F9
:106970002D3239F4689404C00E940435820F911DB1
:10698000219120532A30C0F31EF4909581959F4F9A
:10699000089591110C948336803219F089508550F6
:1069A000C8F70895FA01A191B081009719F41097E2
:1069B000E1F0CD01DC01CD010D90002011F4C0010A
:1069C00013C0FB012191222319F02015D9F7F3CF31
:1069D000FB012191201519F41E92119606C0222365
:1069E000C1F70D900020A1F7D001FA01A193B08367
:1069F0000895BB274A3031F4992322F4BDE29095E3
:106A000081959F4F0C940D357AE0979F902D879F2D
:106A1000802D910D11240895BB27FB015527AA272E
:106A2000880F991FAA1FA41710F0A41B839550511B
:106A3000B9F7A05DAA3308F0A95DA193009779F793
:106A4000B111B1931192CB010C949E36A0E0B0E04D
:106A5000ECE2F5E30C945038EC017B016115710513
:106A600019F0DB018D939C938E010F5F1F4F78808F
:106A7000872D90E00E94C934892B11F0E801F4CFF2
:106A8000BDE27B1205C00F5F1F4F7980C1E008C0D7
:106A9000EBE27E1204C08E010E5F1F4F7980C0E0D2
:106AA0006801F1E0CF1AD10843E050E06EE770E0F2
:106AB000C6010E948636892BF1F4680122E0C20EDD
:106AC000D11C45E050E069E770E0C6010E948636BF
:106AD000892B21F4680187E0C80ED11CE114F10470
:106AE00019F0D701CD92DC92C111FFC060E070E0D7
:106AF00080E89FE703C143E050E066E770E0C6012D
:106B00000E948636892B51F4E114F10409F4F2C095
:106B10000E5F1F4FF70111830083ECC0680160E036
:106B200070E0CB0100E010E0F601D0EDD70DDA30D7
:106B300058F52C2F2260622E2C2F2870C2FF05C022
:106B4000211128C00F5F1F4F25C0222311F00150D3
:106B50001109A5E0B0E09B01AC010E9439384B015E
:106B60005C01880C991CAA1CBB1CC501B4016D0FEB
:106B7000711D811D911D6839A9E97A078A07A9E16C
:106B80009A0740F0C66005C0DE3F51F4C3FD44C023
:106B9000C8606C2EBFEFCB1ADB0A7080C62DC4CF45
:106BA0002D2F2F7D2531C1F540814D3211F4C0616B
:106BB00006C04B3221F0319621E030E006C032961B
:106BC000D60111964C9122E030E0A0EDA40FAA303E
:106BD00018F0E21BF30B20C040E050E04038BCE06E
:106BE0005B075CF49A01220F331F220F331F420F01
:106BF000531F440F551F4A0F511D3196DF01119746
:106C00002C91A0EDA20FAA3048F3C4FF03C0519508
:106C100041955109040F151FC1FF07C0E114F1048C
:106C200021F03197D701ED93FC930E94B336C370E6
:106C3000C33019F06B017C0106C06B017C01F7FACF
:106C4000F094F7F8F09420E030E0A901C701B60114
:106C50000E94AE36882309F445C017FF06C011957F
:106C600001951109C5E9D0E002C0CDEAD0E05E018E
:106C7000B8E1AB1AB1084601BE2DAF2D90E2E92E66
:106C8000F12C0E151F0584F0FE01259135914591DB
:106C90005491B4018B2F9A2F0E9414374B01B82FB7
:106CA000A92F0E191F09EDCF2497F594E794CA1563
:106CB000DB0539F76401EB2EFA2E8E2D880F8F2D10
:106CC000881F8F3F49F020E030E0A901C701B601DD
:106CD0000E94AE36811106C082E290E09093C70612
:106CE0008093C606C701B60109C060E070E080E885
:106CF0009FEF04C060E070E080EC9FE7CDB7DEB7A7
:106D0000EEE00C946C38992788270895FB01DC018C
:106D10004150504088F08D9181341CF08B350CF43B
:106D2000805E659161341CF06B350CF4605E861BEF
:106D3000611171F3990B0895881BFCCFDC01FC01F4
:106D4000672F71917723E1F7329704C07C916D939F
:106D500070836291AE17BF07C8F308950E94F036A2
:106D600008F481E00895E89409C097FB3EF49095FB
:106D70008095709561957F4F8F4F9F4F9923A9F014
:106D8000F92F96E9BB279395F695879577956795A3
:106D9000B795F111F8CFFAF4BB0F11F460FF1BC0E7
:106DA0006F5F7F4F8F4F9F4F16C0882311F096E97A
:106DB00011C0772321F09EE8872F762F05C0662328
:106DC00071F096E8862F70E060E02AF09A95660FE1
:106DD000771F881FDAF7880F9695879597F908959A
:106DE000990F0008550FAA0BE0E8FEEF16161706DC
:106DF000E807F907C0F012161306E407F50798F044
:106E0000621B730B840B950B39F40A2661F0232B5C
:106E1000242B252B21F408950A2609F4A140A695D8
:106E20008FEF811D811D08950E9427370C9498379C
:106E30000E948A3738F00E94913720F0952311F094
:106E40000C9481370C94873711240C94CC370E9412
:106E5000A93770F3959FC1F3950F50E0551F629FBE
:106E6000F001729FBB27F00DB11D639FAA27F00DA3
:106E7000B11DAA1F649F6627B00DA11D661F829FCA
:106E80002227B00DA11D621F739FB00DA11D621FAF
:106E9000839FA00D611D221F749F3327A00D611DCC
:106EA000231F849F600D211D822F762F6A2F1124AE
:106EB0009F5750409AF0F1F088234AF0EE0FFF1FE1
:106EC000BB1F661F771F881F91505040A9F79E3F38
:106ED000510580F00C9481370C94CC375F3FE4F37C
:106EE000983ED4F3869577956795B795F795E7958E
:106EF0009F5FC1F7FE2B880F911D9695879597F997
:106F0000089597F99F6780E870E060E008959FEF2B
:106F100080EC089500240A94161617061806090630
:106F2000089500240A9412161306140605060895FF
:106F3000092E0394000C11F4882352F0BB0F40F487
:106F4000BF2B11F460FF04C06F5F7F4F8F4F9F4FC7
:106F5000089557FD9058440F551F59F05F3F71F049
:106F60004795880F97FB991F61F09F3F79F08795B0
:106F70000895121613061406551FF2CF4695F1DF39
:106F800008C0161617061806991FF1CF86957105C9
:106F9000610508940895E894BB2766277727CB01FD
:106FA00097F90895F999FECF92BD81BDF89A992776
:106FB00080B50895262FF999FECF1FBA92BD81BDE5
:106FC00020BD0FB6F894FA9AF99A0FBE019608956B
:106FD000DB018F939F930E943938BF91AF91A29F9D
:106FE000800D911DA39F900DB29F900D11240895C7
:106FF000A1E21A2EAA1BBB1BFD010DC0AA1FBB1FBD
:10700000EE1FFF1FA217B307E407F50720F0A21B2E
:10701000B30BE40BF50B661F771F881F991F1A949B
:1070200069F760957095809590959B01AC01BD01C5
:10703000CF010895052E97FB1EF400940E9431386D
:1070400057FD07D00E94F83707FC03D04EF40C948C
:10705000313850954095309521953F4F4F4F5F4FB8
:10706000089590958095709561957F4F8F4F9F4FB4
:1070700008950E948338A59F900DB49F900DA49F02
:10708000800D911D11240895B7FF0C9439380E948A
:107090003938821B930B08952F923F924F925F9243
:1070A0006F927F928F929F92AF92BF92CF92DF9218
:1070B000EF92FF920F931F93CF93DF93CDB7DEB77D
:1070C000CA1BDB0B0FB6F894DEBF0FBECDBF099411
:1070D0002A88398848885F846E847D848C849B8468
:1070E000AA84B984C884DF80EE80FD800C811B8176
:1070F000AA81B981CE0FD11D0FB6F894DEBF0FBEA5
:10710000CDBFED010895A29FB001B39FC001A39F21
:10711000700D811D1124911DB29F700D811D1124D0
:10712000911D08955058BB27AA270E94AA380C9495
:1071300098370E948A3738F00E94913720F039F44E
:107140009F3F19F426F40C9487370EF4E095E7FB83
:107150000C948137E92F0E94A93758F3BA176207B8
:1071600073078407950720F079F4A6F50C94CB37C4
:107170000EF4E0950B2EBA2FA02D0B01B901900152
:107180000C01CA01A0011124FF27591B99F0593F96
:1071900050F4503E68F11A16F040A22F232F342FDE
:1071A0004427585FF3CF469537952795A795F0402C
:1071B0005395C9F77EF41F16BA0B620B730B840B41
:1071C000BAF09150A1F0FF0FBB1F661F771F881FF9
:1071D000C2F70EC0BA0F621F731F841F48F4879551
:1071E00077956795B795F7959E3F08F0B0CF939543
:1071F000880F08F09927EE0F9795879508950E94BC
:1072000013390C9498370E94913758F00E948A37AE
:1072100040F029F45F3F29F00C94813751110C9410
:10722000CC370C9487370E94A93768F39923B1F3C0
:10723000552391F3951B550BBB27AA27621773079C
:10724000840738F09F5F5F4F220F331F441FAA1F30
:10725000A9F335D00E2E3AF0E0E832D091505040EC
:10726000E695001CCAF72BD0FE2F29D0660F771F9A
:10727000881FBB1F261737074807AB07B0E809F080
:10728000BB0B802DBF01FF2793585F4F3AF09E3F05
:10729000510578F00C9481370C94CC375F3FE4F3C0
:1072A000983ED4F3869577956795B795F7959F5F48
:1072B000C9F7880F911D9695879597F90895E1E094
:1072C000660F771F881FBB1F621773078407BA07F3
:1072D00020F0621B730B840BBA0BEE1F88F7E0954E
:1072E00008950E9478396894B1110C94CC370895B0
:1072F0000E94B13788F09F5798F0B92F9927B7515E
:10730000B0F0E1F0660F771F881F991F1AF0BA9549
:10731000C9F714C0B13091F00E94CB37B1E00895A5
:107320000C94CB37672F782F8827B85F39F0B93F97
:10733000CCF3869577956795B395D9F73EF49095FC
:107340008095709561957F4F8F4F9F4F08950E9454
:10735000F03608F48FEF08950E94F036880B990BF1
:107360000895EE0FFF1F0590F491E02D0994692711
:1073700096276927782787277827089581E090E066
:10738000F8940C94053A9111089581568A5108F4A5
:10739000805285580895FB01DC0104C08D91019055
:1073A000801921F441505040C8F7881B990B08956B
:1073B000DC0101C06D9341505040E0F70895FB019E
:1073C000DC010D900020E9F7119701900D9200204B
:1073D000E1F70895FC018191861721F08823D9F700
:1073E000992708953197CF010895FB01DC018D9114
:1073F000019080190110D9F3990B0895FB01DC016C
:0E74000001900D920020E1F70895F894FFCF5F
:10740E00B80B1715171501FFFF0A000101FF88744D
:10741E0069692D3035C0A800B42F412D474D2F611D
:10742E00676D2E7068700000000000000000000004
:10743E0000000000000000000000000F27010A8C71
:10744E00CDCC194300C001010000001E004B009678
:10745E00009001E803D00701005E0000000000006C
:10746E00003115311599253115311531153115317B
:10747E001501103115311531153115311531153103
:10748E00153115311500000000CC0F2D109925E592
:10749E000BE20F620EB50DED103C0FD810B6116554
:1074AE00106D118B0E430EFA0FEA0FE60F0000005F
:1074BE00005614C313EE139D141F14FD1311140064
:1074CE00000000160CE60B99252215DD0BC90B23C7
:1074DE001500000000DB0CC3139925982500000051
:1074EE0000311531159925311531153115311531FB
:1074FE0015311531153115311531150000000031DA
:10750E0015C3139925982531153115311500000035
:10751E00007325412699252C10BA25A0251A11B5E0
:10752E0026C3259C258F126B1224109525932519A1
:10753E00108925000000000310521399259825FE8E
:10754E0011000000003115C3139925982500000085
:10755E0000BC15000000003115000040001400545E
:10756E0000312E33000D0A004A756E203130203264
:10757E003031390031333A32393A3331003F002657
:10758E00003A30003A0020446179202D200043500B
:10759E004D3D004D41583D00544F543D004156471E
:1075AE003D00454C503D005245534554004D41431E
:1075BE000055524C00454550524F4D004A534F4EC8
:1075CE0000496E76616C696421006E616E00696EB1
:0E75DE0066006F766600435F474D5F5F0000FA
:107800000C94343C0C94513C0C94513C0C94513CE1
:107810000C94513C0C94513C0C94513C0C94513CB4
:107820000C94513C0C94513C0C94513C0C94513CA4
:107830000C94513C0C94513C0C94513C0C94513C94
:107840000C94513C0C94513C0C94513C0C94513C84
:107850000C94513C0C94513C0C94513C0C94513C74
:107860000C94513C0C94513C11241FBECFEFD8E036
:10787000DEBFCDBF11E0A0E0B1E0ECE9FFE702C060
:1078800005900D92A230B107D9F712E0A2E0B1E065
:1078900001C01D92AD30B107E1F70E942D3D0C945F
:1078A000CC3F0C94003C982F959595959595959582
:1078B000905D8F708A307CF0282F295A8091C0000B
:1078C00085FFFCCF9093C6008091C00085FFFCCF60
:1078D0002093C6000895282F205DF0CF982F809127
:1078E000C00085FFFCCF9093C6000895EF92FF92F1
:1078F0000F931F93EE24FF2487018091C00087FD22
:1079000017C00894E11CF11C011D111D81E4E8164B
:1079100082E4F8068FE0080780E0180770F3E09132
:107920000401F091050109958091C00087FFE9CF1E
:107930008091C6001F910F91FF90EF9008950E94D3
:10794000763C982F8091C00085FFFCCF9093C600B5
:1079500091362CF490330CF09053892F089597555D
:10796000892F08951F930E949F3C182F0E949F3CCF
:107970001295107F810F1F9108951F93182F882350
:1079800021F00E94763C1150E1F71F9108951F935A
:10799000182F0E94763C803249F0809103018F5F5E
:1079A000809303018530C1F01F9108958091C0003C
:1079B00085FFFCCF84E18093C6008091C00085FFE5
:1079C000FCCF1093C6008091C00085FFFCCF80E102
:1079D0008093C6001F910895E0910401F091050184
:1079E00009951F9108950E94763C803241F0809164
:1079F00003018F5F80930301853081F008958091AA
:107A0000C00085FFFCCF84E18093C6008091C00058
:107A100085FFFCCF80E18093C6000895E0910401CA
:107A2000F09105010995089540E951E08823A1F0FE
:107A30002D9A28EE33E0FA013197F1F721503040CA
:107A4000D1F72D9828EE33E0FA013197F1F7215064
:107A50003040D1F7815061F708953F924F925F9285
:107A60006F927F928F929F92AF92BF92CF92DF924E
:107A7000EF92FF920F931F93CF93DF93000080E16B
:107A80008093C4001092C50088E18093C10086E015
:107A90008093C2005098589A259A81E00E94143D24
:107AA00024E1F22E9EE1E92E85E9D82E0FE0C02ECA
:107AB00010E1B12EAA24A394B1E49B2EA6E58A2E50
:107AC000F2E57F2EE0E26E2E79E4572E63E5462E36
:107AD00050E5352E0E94763C8033B1F18133B9F107
:107AE000803409F46FC0813409F476C0823409F41B
:107AF00085C0853409F488C0803531F1823521F1A3
:107B0000813511F1853509F485C0863509F48DC0BC
:107B1000843609F496C0843709F403C1853709F423
:107B200072C1863709F466C0809103018F5F80932C
:107B30000301853079F6E0910401F0910501099582
:107B40000E94763C803351F60E94F33CC3CF0E94E2
:107B5000763C803249F78091C00085FFFCCFF092DF
:107B6000C6008091C00085FFFCCF9092C600809136
:107B7000C00085FFFCCF8092C6008091C00085FFC9
:107B8000FCCF7092C6008091C00085FFFCCF609250
:107B9000C6008091C00085FFFCCF5092C600809146
:107BA000C00085FFFCCF4092C6008091C00085FFD9
:107BB000FCCF3092C6008091C00085FFFCCFB09210
:107BC000C60088CF0E94763C863808F4BDCF0E945C
:107BD000763C0E94F33C7ECF0E94763C803809F4CC
:107BE0009CC0813809F40BC1823809F43CC1883942
:107BF00009F48FC080E00E94C73C6CCF84E10E94F2
:107C0000BD3C0E94F33C66CF85E00E94BD3C0E94D3
:107C1000F33C60CF0E94763C809306010E94763C44
:107C2000809307010E94F33C55CF0E94763C80333D
:107C300009F41DC183E00E94BD3C80E00E94C73C66
:107C400049CF0E94763C809309020E94763C809343
:107C5000080280910C028E7F80930C020E94763C79
:107C6000853409F415C18091080290910902892B8D
:107C700089F000E010E00E94763CF801E85FFE4FDA
:107C800080830F5F1F4F80910802909109020817AF
:107C9000190788F30E94763C803209F045CF809125
:107CA0000C0280FF01C16091060170910701660F0F
:107CB000771F7093070160930601A0910802B091AD
:107CC00009021097C9F0E8E0F1E09B01AD014E0F09
:107CD0005F1FF999FECF32BD21BD819180BDFA9A17
:107CE000F99A2F5F3F4FE417F50799F76A0F7B1F4B
:107CF00070930701609306018091C00085FFFCCF5F
:107D0000F092C6008091C00085FFFCCFB092C60003
:107D1000E1CE83E00E94C73CDDCE82E00E94C73CFA
:107D2000D9CE0E94763C809309020E94763C8093D3
:107D300008028091060190910701880F991F909386
:107D40000701809306010E94763C853409F4A6C0A1
:107D500080910C028E7F80930C020E94763C8032D0
:107D600009F0B8CE8091C00085FFFCCFF092C6002C
:107D7000609108027091090261157105B9F140E046
:107D800050E080910C02A82FA170B82FB27011C0E2
:107D9000BB2309F45CC0E0910601F0910701319624
:107DA000F0930701E09306014F5F5F4F46175707B7
:107DB000E8F4AA2369F3F999FECF209106013091E6
:107DC000070132BD21BDF89A90B58091C00085FFB2
:107DD000FCCF9093C6002F5F3F4F30930701209355
:107DE00006014F5F5F4F4617570718F38091C00099
:107DF00085FDE5CE8091C00085FFF8CFE0CE81E023
:107E00000E94C73C67CE0E94763C803209F08CCE3F
:107E10008091C00085FFFCCFF092C6008091C00029
:107E200085FFFCCFE092C6008091C00085FFFCCFAB
:107E3000D092C6008091C00085FFFCCFC092C600E2
:107E40008091C00085FFFCCFB092C60043CEE09188
:107E50000601F091070194918091C00085FFFCCF4D
:107E60009093C6009CCF80E10E94C73C33CE0E9415
:107E7000763C0E94763C182F0E94763C112309F430
:107E800083C0113009F484C08FE00E94C73C22CE29
:107E900080910C02816080930C02E5CE80910C02EF
:107EA000816080930C0259CF809107018823880F4D
:107EB000880B8A2180930B02809106019091070123
:107EC000880F991F90930701809306018091080203
:107ED00080FF09C080910802909109020196909359
:107EE000090280930802F894F999FECF1127E091D6
:107EF0000601F0910701C8E0D1E08091080290915D
:107F00000902103091F40091570001700130D9F34B
:107F100003E000935700E89500915700017001308D
:107F2000D9F301E100935700E89509901990009169
:107F3000570001700130D9F301E000935700E89534
:107F40001395103498F011270091570001700130FB
:107F5000D9F305E000935700E895009157000170B0
:107F60000130D9F301E100935700E895329602976A
:107F700009F0C7CF103011F00296E5CF112480919F
:107F8000C00085FFB9CEBCCE8EE10E94C73CA2CD19
:0C7F900085E90E94C73C9ECDF894FFCF0D
:027F9C00800063
:040000030000780081
:00000001FF
